:020000040800F2
:10000000C08C0020BD010008C5010008C701000820
:10001000C9010008CB010008CD0100080000000064
:10002000000000000000000000000000CF010008F8
:10003000D101000800000000D3010008D50100082C
:10004000D7010008D7010008D7010008D701000830
:10005000D7010008D7010008D7010008D701000820
:10006000D7010008D7010008D7010008D701000810
:10007000D7010008D7010008F93F0008D7010008A0
:10008000D7010008D7010008D701000800000000D0
:10009000000000000000000000000000D701000880
:1000A000D7010008D7010008D7010008D7010008D0
:1000B0000D28000821300008D7010008D7010008EA
:1000C000D7010008D7010008D7010008D7010008B0
:1000D000D701000805410008D7010008574600086D
:1000E000D7010008D7010008D70100080000000070
:1000F0000000000000000000000000000000000000
:1001000000000000000000000000000000000000EF
:100110000000000000000000D7010008D70100081F
:1001200000F002F800F03AF80AA090E8000C8244CF
:100130008344AAF10107DA4501D100F02FF8AFF2AC
:10014000090EBAE80F0013F0010F18BFFB1A43F0B5
:10015000010318472443010044430100103A24BF1F
:1001600078C878C1FAD8520724BF30C830C144BF1C
:1001700004680C607047000000230024002500265E
:10018000103A28BF78C1FBD8520728BF30C148BFFA
:100190000B6070471FB51FBD10B510BD04F02AFEDF
:1001A0001146FFF7F7FF02F09FF904F048FE03B491
:1001B000FFF7F2FF03BC04F04BFE00000948804744
:1001C00009480047FEE7FEE7FEE7FEE7FEE7FEE739
:1001D000FEE7FEE7FEE7FEE704480549054A064B51
:1001E000704700003524000821010008C086002067
:1001F000C08C0020C0880020C08800202849084307
:1002000028490860704770B50F23C478017801222F
:10021000F4B1244C2468457804F4E064C4F5E06447
:10022000240AC4F10406E3408478B5401C402C4302
:1002300001F1E021230181F80034007800F01F0172
:100240008A404009800000F1E020C0F8002170BD24
:1002500001F01F0082404809800000F1E020C0F852
:10026000802170BD104A114001430E48001F0160FB
:1002700070470C4A121D0029116801D0014300E0AB
:100280008143116070474FF0E0210428086903D0D2
:1002900020F004000861704740F00400FAE7000015
:1002A0000000FA050CED00E080FFFF1FC54910B506
:1002B000884202D1012144150AE0C349884202D193
:1002C0000121041504E0C14988420AD10121CC036F
:1002D000204601F08CF82046BDE81040002101F0D6
:1002E00086B810BD10B54268B94B0C791A400B683E
:1002F00042EA0422134343608368B64A1340D1E9BB
:10030000024222434C7943EA44031A438260C26AA0
:10031000097C22F47002491EC9B242EA0151C1624D
:1003200010BD00210160017141718160C160012136
:10033000017470470029816802D041F0010101E099
:1003400021F00101816070470029816802D041F4E9
:10035000807101E021F4807181607047002A426859
:10036000C9B201D00A4300E08A4342607047816805
:1003700041F0080181607047014600208968090743
:1003800000D501207047816841F004018160704709
:10039000014600208968490700D5012070470029DF
:1003A000816802D041F4A00101E021F4A001816044
:1003B0007047014600208968490200D50120704736
:1003C0004268491E22F4604242EA4131416070476E
:1003D0000029416802D041F4006101E021F400618C
:1003E0004160704770B5072409290AD9C568A1F191
:1003F0000A0606EB4606B440A543B3401D43C5605C
:1004000007E0056901EB4106B440A543B3401D4335
:1004100005611F23072A09D2446B521E02EB820298
:1004200093409C4391400C43446370BD0D2A09D214
:10043000046BD21F02EB820293409C4391400C4319
:10044000046370BDC46A0D3A02EB820293409C4380
:1004500091400C43C46270BD0029816802D041F410
:10046000801101E021F4801181607047C06C80B27E
:10047000704754484C30006870470029416802D0EA
:1004800041F4806101E021F48061416070470029FE
:10049000416802D041F4805101E021F48051416073
:1004A0007047826822F4E0420A4382607047002964
:1004B000816802D041F4004101E021F400418160F3
:1004C00070470029816802D041F4021101E021F453
:1004D000021181607047014600208968890200D5B9
:1004E0000120704770B5072409290AD9C568A1F110
:1004F0000A0606EB4606B440A543B3401D43C5605B
:1005000007E0056901EB4106B440A543B3401D4334
:100510000561836BC3F30154121B921C02EB82042E
:100520001F22A2409343A1400B43836370BD826BA3
:10053000491E22F4401242EA01518163704708B516
:1005400008440090026008BD08B5084428300090B7
:10055000006880B208BD42681F4B1A400A434260DF
:100560007047416282627047426822F01F020A436C
:1005700042607047134908310028086802D040F4EF
:10058000000001E020F400000860704702460020EF
:1005900012680A4200D001207047C94301607047C9
:1005A00010B50246002054680B0AC9B20C4011680D
:1005B000194202D0002C00D0012010BD6FEA112199
:1005C000016070470024014000280140003C0140C8
:1005D000FFFEF0FFFDF7F1FFFFFD3FFF10B501202B
:1005E00000F017FFBDE81040002000F012BF1F49C7
:1005F000086070471D49091F086070471B49843116
:10060000086070471A4A118821F460710143118013
:100610007047174A118821F07F010143118070470C
:10062000134A08B52C3A10440090016008BD1049E7
:1006300008B52C3908440090008808BD0B489C3050
:100640000068C0B270470A480830018841F00101D3
:10065000018070470548A0300068C0B27047044868
:100660000830018841F002010180704704860D4284
:100670002C6C004010B501214C07204600F0C0FE54
:100680002046BDE81040002100F0BABE30B5374C1E
:10069000236840F6FE7282409343D1E900252A4345
:1006A000D1E902510D432A4382401A43226030BDF2
:1006B0000021016041608160C16070472B4A0123C5
:1006C0008340106809B1184300E0984310607047F8
:1006D000264A93148340106809B1184300E09843F8
:1006E00010607047214A121D03090120984000291B
:1006F000116801D0014300E08143116070471B493C
:10070000091D0028086802D040F0030001E020F035
:10071000030008607047154B814018680AB1084310
:1007200000E0884318607047104A08B5104408304C
:100730000090016008BD0D4A08B5104414300090C7
:10074000016008BD082805D042EA0141074A10446B
:100750000162704742EA0121F8E7044908B501EB5C
:1007600090002C300090006880B208BD00740040FA
:1007700001684FF6FE721140016000210160416086
:100780008160C1606A496A4A0839904203D1486869
:1007900040F00F0006E0664A1432904204D14868E7
:1007A00040F0F00048607047614A2832904203D11F
:1007B000486840F47060F5E75D4A3C32904203D1EE
:1007C000486840F47040EDE7594A5032904203D1F6
:1007D000486840F47020E5E7554A6432904203D1FE
:1007E000486840F47000DDE7514A7832904203D106
:1007F000486840F07060D5E74E4A111F904203D11F
:10080000086840F00F0006E04A4A1432904204D1D2
:10081000086840F0F00008607047464A283290426D
:1008200003D1086840F47060F5E7424A3C329042D8
:1008300003D1086840F47040EDE73E4A50329042E0
:10084000EAD1086840F47020E5E730B5036847F660
:10085000F07293430C6A8A682243D1E904452C4321
:1008600022438C692243CC6922434C6A22438C6A1E
:1008700022431A430260CA6842600A68826049687B
:10088000C16030BD0021016041608160C1600161D3
:1008900041618161C16101624162816270470029E9
:1008A000016802D041F0010102E04FF6FE721140F2
:1008B00001607047002A026801D00A4300E08A43C1
:1008C0000260704741607047406880B270470146DF
:1008D0000020CA0002D5174A083A01E0144A083A33
:1008E00012680A4200D001207047C10003D51149A7
:1008F000091F086070470E49083948607047014673
:100900000020CA0002D50B4A083A01E0084A083A1A
:1009100012680A4200D001207047C10003D5054982
:10092000091F086070470249083948607047000095
:100930000800024008040240374900200860091DF1
:100940000860091D0860091D0860334933481431E7
:100950000860704730B530498379026853B30B683B
:1009600093430B600A1D13680468A3431360027964
:100970000A441368046823431360274A0832136843
:100980000468A3431360131D1C680568AC431C6016
:100990004479102C05D021440A68006802430A609B
:1009A00030BD116804682143116019680068014373
:1009B000196030BD0079084401689143016030BD81
:1009C0000021016001710C2242718171704712494E
:1009D00010310A6802430A60704701460E4A00203F
:1009E000143212680A4200D0012070470A491431BB
:1009F00008607047084A014600201268064B0A400A
:100A000014331B680B4202D0002A00D0012070472B
:100A1000014914310860704700040140FFFF0F00D6
:100A2000FC4A116801F03801014311607047F9492F
:100A30000A6822F008020A600A6802430A607047E6
:100A4000F4490A6822F010020A600A6802430A6048
:100A50007047F048F0494160F04941607047ED4807
:100A6000ED494160ED4941607047EA48016941F054
:100A7000800101617047E748016941F0800101612F
:100A80007047E4490420CA68D20701D001207047AA
:100A9000CA68520701D502207047C968C906FBD54C
:100AA0000320704700B50346FFF7EBFF03E000BFEC
:100AB000FFF7E7FF5B1E012803D0002B00D10520C4
:100AC00000BD002BF4D1FAE770B505464FF430268F
:100AD0003046FFF7E7FF042811D1CE4C206940F0E3
:100AE000020020616561206940F0400020613046CD
:100AF000FFF7D8FF216941F6FD721140216170BDF9
:100B000030B54FF430252846FFF7CCFF042810D12C
:100B1000C04C206940F004002061206940F0400092
:100B200020612846FFF7BEFF216941F6FB721140A4
:100B3000216130BD00B50346FFF7A3FF03E000BF0E
:100B4000FFF79FFF5B1E012803D0002B00D105207B
:100B500000BD002BF4D1FAE730B54FF4302528461C
:100B6000FFF7E8FF042810D1AA4C206940F00400E8
:100B70002061206940F0400020612846FFF7DAFF3D
:100B8000216941F6FB721140216130BDA14900206D
:100B9000C969890700D50120704770B5A525FFF701
:100BA000F5FF00B100254FF430263046FFF77AFFFD
:100BB000042827D1974C9848A0609848A0602069E5
:100BC00040F020002061206940F040002061304664
:100BD000FFF768FF41F6EF7604280ED1206941F651
:100BE000DF7108402061206940F0100020618C48CE
:100BF00005804FF40050FFF755FF052802D021690A
:100C00003140216170BDF8B5064600204FF4005C0C
:100C100000900D466046FFF745FF042816D17D4C35
:100C2000206940F00100206135806046FFF73AFFFF
:100C300041F6FE77042806D1B61C280C00963080B9
:100C40006046FFF72FFF216939402161F8BDF0B5FB
:100C500006464FF400570D463846FFF723FF042899
:100C60000CD16C4C206940F0010020613580384681
:100C7000FFF718FF2169BA1E11402161F0BDF0B5E0
:100C800006464FF400570D463846FFF70BFF042881
:100C900013D1604C6048A0606048A060206940F0BB
:100CA0001000206135803846FFF7FCFE052804D08F
:100CB000216941F6EF7211402161F0BD2DE9F0414B
:100CC000C04300F0FF0CC0F30727C0F30746050E32
:100CD0004FF400584046FFF7E5FE042837D14D4C4D
:100CE0004D49A1604D49A160216941F01001216188
:100CF000BCF1FF0F08D04A480830A0F800C04046B9
:100D0000FFF7D0FE04281BD1FF2F07D044480A303C
:100D100007804046FFF7C6FE042811D1FF2E07D0FA
:100D20003F480C3006804046FFF7BCFE042807D140
:100D3000FF2D07D03A480E3005804046FFF7B2FE3F
:100D4000052804D0216941F6EF7211402161BDE808
:100D5000F08170B505464FF430263046FFF7A2FE0D
:100D6000042818D12B4C2C48A0602C48A060206986
:100D700040F020002061206940F0400020613046B2
:100D8000FFF790FE41F6DF71042805D0052802D058
:100D900022690A40226170BD2069084020612069F3
:100DA00040F0100020611E480DB1002100E0A52197
:100DB00001803046FFF776FE0528ECD0216941F628
:100DC000EF721140216170BDF0B5124C0746124818
:100DD00016460D46A0601148A0604FF4005C6046C6
:100DE000FFF760FE042814D1206940F01000206154
:100DF00035430B493D43891C45F0F80008806046A7
:100E0000FFF750FE052804D0216941F6EF7211402A
:100E10002161F0BD0020024023016745AB89EFCD81
:100E200000F8FF1F1C48C069800870471A48006A14
:100E30007047194900200968890600D501207047CC
:100E4000154A0029116901D0014300E08143116175
:100E5000704701460020104A012903D0D2680A4297
:100E600003D17047D169C907FBD0012070470A49F7
:100E7000C860704708490420CA68D20701D0012021
:100E80007047CA68520701D502207047C968C90671
:100E9000FBD503207047000000200240914910B5A7
:100EA000884206D10121042000F0A1FA002104208B
:100EB0003BE08D49884206D10121082000F097FAD5
:100EC0000021082031E08949884206D10121102003
:100ED00000F08DFA0021102027E08549884206D1D4
:100EE0000121202000F083FA002120201DE081490B
:100EF000884206D10121402000F079FA00214020EB
:100F000013E07D49884206D10121802000F06FFA6C
:100F10000021802009E0794988420AD18415012105
:100F2000204600F064FA00212046BDE8104000F0A1
:100F30005EBA10BD10B50121084600F058FA002134
:100F4000BDE81040012000F052BAF0B5CA78002583
:100F500002F00F03D20601D58A7813430A784FF0C6
:100F60000F0E12F0FF0F4FF001021DD0D0F800401D
:100F70000F8802FA05F63740B74211D14FEA850CC7
:100F80000EFA0CF724EA070703FA0CF43C43CF7877
:100F9000282F02D0482F02D002E0466100E006610F
:100FA0006D1C082DE4D304600C88FF2C1ED9446806
:100FB0005FF0000606F1080702FA07F50F882F40D8
:100FC000AF420FD14FEA860C0EFA0CF7BC4303FA7E
:100FD0000CF73C43CF78282F00D14561CF78482FBC
:100FE00000D10561761C082EE4D34460F0BD4FF6B5
:100FF000FF710180022181700421C1707047024697
:10100000002092680A4200D001207047806880B2B8
:10101000704702460020D2680A4200D00120704783
:10102000C06880B2704701617047416170470AB182
:101030000161704741617047C160704741F480327F
:101040008261816182618169806970472C4B10B532
:101050001A684FF68074224042EA00100843186074
:1010600010BD2849C8617047F0B5254C002801DA49
:10107000E36900E06368420D120185B2C0F30157D5
:101080009540C0F30346032F05D0C2020AD50322C0
:10109000B240934307E023F07062636823F070630B
:1010A000636002E0AB4343F0706201B12A43002861
:1010B00001DAE261F0BD6260F0BD10B58A0721F08F
:1010C00003040F49130F21440F228C689A40944364
:1010D0008C608A68984002438A6010BD0949C1F853
:1010E000DC00704700080140000C01400010014086
:1010F0000014014000180140001C01400020014084
:10110000000001400000204210B501210C072046DC
:1011100000F076F92046BDE81040002100F070B9DB
:101120002149086270472049086170471F4A1168C9
:1011300021F0E0010143116070471B49C1F8A00094
:1011400070471A4B1A6822F0030202431A601848CB
:10115000026842F004020260012905D020BF016844
:1011600021F004010160704730BFF8E70F480168C3
:1011700041F004010160016841F0020101600C4886
:10118000016841F00401016030BF7047074A014621
:10119000002052680A4200D00120704703490A68C3
:1011A00042EA80000860704700000E420070004074
:1011B00010ED00E0A448016841F0010101604168C0
:1011C000A24A114041600168A14A114001600168D2
:1011D00021F480210160416821F4FE0141604FF457
:1011E0001F018160704798490A6822F480320A60C2
:1011F0000A6822F480220A60B0F5803F07D0B0F57B
:10120000802F03D1086840F4A02008607047086868
:1012100040F48030F9E70246002053098A49012B47
:101220000AD0022B0AD0496A02F01F020123934020
:101230000B4200D0012070470968F5E7096AF3E71F
:1012400018B500204FF4A06400903120FFF7E3FFB1
:101250000099491C0091A14201D00028F5D031200D
:10126000FFF7D9FF002800D0012018BD76490A6891
:1012700022F0F80242EAC000086070477549086031
:101280007047714A5368084323F47C131843506035
:1012900070477049086670476B4A516821F0030136
:1012A0000143516070476848406800F00C00704787
:1012B000654A516821F0F001014351607047624A6C
:1012C000516821F4E0610143516070475E494A680A
:1012D00022F4605242EAC000486070475A4A00292E
:1012E000517A01D0014300E081435172704759495E
:1012F000C1F8D8007047544A516821F44041014375
:10130000516070475049002281F8202081F8202048
:10131000012802D0042802D1052081F8200070475E
:101320004D490860704748490A6A02430A6270479B
:10133000494944390860704730B543494A6812F05A
:101340000C03464A03D0042B01D0082B21D00260A5
:101350004A680F23424C03EA1212A35C0268DA4087
:1013600042604B68072505EA1323E35C22FA03F386
:1013700083604B6805EAD323E35CDA40C2604968C6
:10138000032303EA9131231F595CB2FBF1F10161A0
:1013900030BD4A684B6802F470124FF0020413F437
:1013A000803F04EB924202D04B689B0301D52D4B4A
:1013B00000E02A4B5A43CAE7234A0029516901D069
:1013C000014300E08143516170471F4A0029916940
:1013D00001D0014300E08143916170471A4A00291E
:1013E000D16901D0014300E08143D1617047164AC1
:1013F0000029D16801D0014300E08143D1607047EA
:10140000114A0029116901D0014300E081431161B3
:10141000704711494039086070470E49C8647047E9
:101420000949C87170470848416A41F080714162BA
:101430007047054A0146002092680A4200D0012008
:101440007047014988727047001002400000FFF8A1
:10145000FFFFF6FE000042428004424200127A0082
:101460000400002000093D00424A0029118801D0F3
:10147000014300E08143118070473E48001D018810
:1014800041F01001018070473A48001D018821F0A9
:1014900010010180704737481C30008835491831E9
:1014A000098840EA0140704700B50246FFF7E5FFB2
:1014B0003049100C18310880081D02805DF804EBDB
:1014C000E2E700B50246FFF7D8FF2A49C2F303401E
:1014D00008310880081D02805DF804EBD4E700B5F0
:1014E0000246FFF7CAFF2349100C20310880081D6F
:1014F00002805DF804EBC7E71E4810300088000743
:10150000010B1C4814300088084370471948001D1F
:1015100001888906FCD570471648001D018821F016
:101520000801018001880907FCD570470146114A6E
:101530000020121D12880A4200D0012070470D4978
:10154000091D0A8882430A8070470A49091D0988D3
:10155000C2B21140074A1288024202D009B10120EA
:101560007047002070470349091D0A8882430A809A
:101570007047000000280040F94910B5884202D1A8
:101580000121C41486E0B0F1804F09D0F5498842AA
:101590000DD101210220FFF733FF0021022064E07A
:1015A00001210846FFF72CFF002101205DE0EE49F4
:1015B000884206D101210420FFF722FF00210420E8
:1015C00053E0EA49884206D101210820FFF718FFBD
:1015D0000021082049E0E649884206D10121102077
:1015E000FFF70EFF002110203FE0E249884206D1BC
:1015F00001212020FFF704FF0021202035E0DE49F3
:10160000884202D10121441444E0DC49884202D1DD
:101610000121CC043EE0DA49884202D101210C05C7
:1016200038E0D849884202D101214C0532E0D64940
:10163000884206D101214020FFF7E2FE0021402030
:1016400013E0D249884206D101218020FFF7D8FE5D
:101650000021802009E0CE4988420AD18415012169
:101660002046FFF7CDFE00212046BDE81040FFF7E1
:10167000C7BEC849884202D101210C040AE0C6490C
:10168000884202D101214C0404E0C44988420AD1B5
:1016900001218C042046FFF7AAFE2046BDE8104039
:1016A0000021FFF7A4BE10BD30B50288AC4BB24C90
:1016B00098420DD0A0420BD0B0F1804F08D0A94D78
:1016C000A84205D0A84DA84202D0A84DA84203D1F7
:1016D00022F070054A882A43A54DA84206D0A54DA0
:1016E000A84203D022F44075CA882A4302808A881F
:1016F00082850A88028598420AD0A04208D0A54A6D
:10170000904205D0A44A904202D0A44A904201D10E
:10171000097A01860121818230BD30B5028C22F028
:1017200001020284028C8388048B22F0020224F0DE
:1017300073050C882C430D8915434A882A43884D2C
:10174000A8420BD08C4DA84208D0924DA84205D09B
:10175000914DA84202D0914DA8420DD122F008052A
:101760004A8923F440732A4322F004058A882A43D5
:101770008D891D43CB892B4383800483C98881864F
:10178000028430BD70B5028C22F010020284028CFB
:101790008488038B0D8823F4E6464FF6FF7303EA33
:1017A000052535430E8922F0200203EA061616436A
:1017B0004A8803EA02123243694EB04202D06E4EAA
:1017C000B04215D122F080064A8924F4406403EA2D
:1017D0000212324322F040068A8803EA02123243A0
:1017E0008E8903EA86062643CC8903EA84043443BF
:1017F00084800583C9880187028470BD70B5028C1E
:1018000022F480720284028C8488838B0D8823F0FA
:1018100073031D4322F400730E894FF6FF7202EA30
:1018200006261E434B8802EA032333434C4EB04244
:1018300002D0514EB04215D123F400664B8924F4F6
:10184000405402EA0323334323F480668B8802EA80
:10185000032333438E8902EA06162643CC8902EA23
:101860000414344384808583C9888187038470BDD0
:1018700070B5028C22F480520284048C8288838B9F
:101880000D8823F4E6464FF6FF7303EA052535433A
:1018900024F400560C8903EA043434434E8803EAE6
:1018A000063626432E4CA04202D0334CA04205D12E
:1018B00022F480448A8903EA82122243828085834B
:1018C000C988A0F84010068470BD828B22F4406263
:1018D0008283828B4FF6FF7303EA01210A438283DE
:1018E0007047828B22F00C028283828B0A438283B0
:1018F0007047028B22F440620283028B4FF6FF7323
:1019000003EA01210A4302837047F0B5048C24F0F6
:1019100010040484078B048C4FF6FF7527F473477B
:1019200005EA03333B4305EA02221A430C4B05EA5E
:10193000011698420ED0104B98420BD0B0F1804F58
:1019400008D0084B984205D0074B984202D0074B6D
:10195000984225D124F02001314341F0100124E0C8
:10196000002C01400004004000080040000C004032
:10197000001000400014004000340140004C0140C1
:10198000005001400054014000180040001C00407D
:101990000020004000400140004401400048014058
:1019A00024F0A0030B4343F0100102830184F0BD37
:1019B000028B22F00C020283028B0A4302837047DF
:1019C00070B5048C24F001040484058B048C4FF65C
:1019D000FF7606EA0313134325F0F305F94A2B4378
:1019E00090420ED0F84A90420BD0B0F1804F08D010
:1019F000F64A904205D0F64A904202D0F54A90420B
:101A000002D124F0020201E024F00A020A4342F06B
:101A100001010383018470BD2DE9F05F0D4604468A
:101A20000888E84FDFF8A0C3DFF8A0834988AA88B8
:101A30002B894FF0804960B3042832D04FF6FF7EE7
:101A4000082836D0208C9B4620F480502084A38B1D
:101A5000268C704600EA022223F473431A4300EAFC
:101A60000B3010430EEA013EBC420BD0644509D056
:101A70004C4507D0444505D0D54A944202D0D54BB9
:101A80009C4245D126F4005141EA0E0141F48051B7
:101A900043E02046FFF794FFE9882046BDE8F05F69
:101AA00086E72046FFF731FFE9882046BDE8F05F72
:101AB0001FE7208C20F480702084B4F81CA0208CB8
:101AC0000EEA031313432AF0F30A0EEA012B43EA4A
:101AD0000A03BC420BD0644509D04C4507D04445AD
:101AE00005D0BB4A944202D0BA4A944204D120F4B1
:101AF000007040EA0B0002E020F42060084340F44C
:101B00008070A3832084E9882046BDE8F05FE8E682
:101B100026F402420A4342F48051A08320462184E5
:101B2000E988BDE8F05FD0E62DE9F0410C460026DB
:101B300049880746012501B90226A288012A00D159
:101B40000225208823890028384610D0FFF7DDFEC3
:101B5000E1883846FFF7CDFE23892A4631463846CC
:101B6000FFF72EFFE1883846BDE8F04120E7FFF798
:101B700027FFE1883846FFF71BFF23892A463146B5
:101B80003846FFF7C2FEE1883846BDE8F041B0E6CE
:101B900010B50A884B88CC881A438B8823431A4394
:101BA0000B891A434B8989891A430A43A0F84420B8
:101BB00010BD4FF6FF71818000210180C1804180FE
:101BC000017270470021018041808180C1800181C4
:101BD00041818181C18170470021018041800122C2
:101BE0008280C18001817047002101804180818015
:101BF000C18001814181818170470029018802D023
:101C000041F0010101E021F001010180704700294C
:101C100030F8441F02D041F4004101E0C1F30E014D
:101C200001807047002A828901D00A4300E08A437C
:101C300082817047818270471143A0F84810704735
:101C4000002A828901D00A4300E08A4382817047DA
:101C5000018921F0070101817047028922F0700299
:101C60000A430281704700B50346FFF7F6FF188963
:101C700040F00700188100BD70B516460D4660297A
:101C800004464FF0010231460AD0FFF799FE29467B
:101C90002046FFF7E2FF208940F00700208170BD59
:101CA000FFF733FEF3E730B504894FF6FF7505EA19
:101CB00003231343E4B20B432343038130BD10B528
:101CC0000446FFF7F0FF208940F07700208110BD27
:101CD00010B50446FFF7E7FF208940F480402081DB
:101CE00010BD018582827047028822F070020A438B
:101CF0000280704770B50589048B068C25F00705B6
:101D00000D434FF6FC410C4040F201110C434FF6DD
:101D1000FF7101EA031126F02206114331430581C8
:101D20000483018470BD028B22F070020A43028397
:101D30007047028B4FF6FF7322F4E04203EA012161
:101D4000114301837047828B22F070020A43828321
:101D50007047828B4FF6FF7322F4E04203EA0121C1
:101D60001143818370470029018802D041F080012E
:101D700001E021F08001018070470029818802D0B4
:101D800041F0040101E021F0040181807047002945
:101D9000818802D041F0080101E021F00801818032
:101DA00070470029818802D041F0010101E021F053
:101DB000010181807047028B22F008020A430283EE
:101DC00070470000002C0140003401400004004036
:101DD00000080040000C0040028B4FF6FF7322F415
:101DE000006203EA012111430183E9E7828B22F0BB
:101DF00008020A438283E3E7828B4FF6FF7322F4E3
:101E0000006203EA012111438183D9E7028B22F0AA
:101E100004020A430283D3E7028B4FF6FF7322F4D6
:101E2000806203EA012111430183C9E7828B22F01A
:101E300004020A438283C3E7828B4FF6FF7322F4C6
:101E4000806203EA012111438183B9E7028B22F00A
:101E500080020A430283B3E7028B4FF6FF73C2F39B
:101E60000E0203EA012111430183A9E7828B22F0CC
:101E700080020A438283A3E7828B4FF6FF73C2F38B
:101E80000E0203EA01211143818399E7028C22F0BB
:101E900002020A43028493E7028C22F008020A43FA
:101EA00002848DE7028C4FF6FF7322F0200203EAD2
:101EB00001111143018483E7028C4FF6FF7322F076
:101EC000800203EA01111143018479E7028C4FF685
:101ED000FF7322F4007203EA0121114301846FE7CA
:101EE000028C4FF6FF7322F4006203EA01211143D2
:101EF000018465E7028C4FF6FF7322F4005203EA77
:101F00000131114301845BE710B50123048C8B4040
:101F10009C430484038C8A401343038410BD10B592
:101F20000423048C8B409C430484038C8A40134319
:101F3000038410BD30B50124058C00F118038C40DA
:101F4000A543058489B108290FD0091FC1F34E00AC
:101F50001844016821F4E041016001684FF6FF7305
:101F600003EA02221143016030BD03EB5100016816
:101F700021F0700101600168F4E70029018802D0B6
:101F800041F0020101E021F00201018018E700297F
:101F9000018802D041F0040101E021F00401018038
:101FA0000EE70029818802D041F0800101E021F094
:101FB0008001818004E7028822F008020280028802
:101FC0000A430280FCE6828822F0700282808288C6
:101FD0000A438280F4E6028922F007020281028924
:101FE0000A430281ECE6028922F080020281028922
:101FF0000A430281E4E68184E2E68185E0E68186A7
:10200000DEE60187DCE68187DAE6A0F84010D7E655
:10201000028822F44072028002880A430280CFE6DE
:10202000808ECDE6008FCBE6808FC9E6B0F8400009
:10203000C6E6808CC4E6008DC2E602460020128A05
:102040000A4200D00120BBE6C9430182B8E602463D
:102050000020138A92890B4202EA010202D0002A70
:1020600000D00120ACE6C9430182A9E6C44910B5FD
:1020700088420AD101218C032046FFF7B8F9204697
:10208000BDE810400021FFF7B2B9BE49884202D135
:1020900001214C0410E0BC49884202D101218C048A
:1020A0000AE0BA49884202D10121CC0404E0B849CF
:1020B00088420AD101210C052046FFF7A1F92046EC
:1020C000BDE810400021FFF79BB910BD30B50446B4
:1020D000008A85B00D464CF6FF710840E98801433F
:1020E0002182A1894EF6F3100140A8882A89104365
:1020F0006A890A431043A081A08A4FF6FF41084035
:10210000A9890143A1826846FFF716F99C488442D9
:1021100001D1039800E00298A189090400EBC001F5
:1021200001EB0010296801D5490000E08900B0FBEF
:10213000F1F06422B0FBF2F109010B096FF0180510
:102140006B4300EB8300A3891D044FF0320306D5D7
:1021500003EBC000B0FBF2F000F0070005E003EB7A
:102160000010B0FBF2F000F00F000843208105B032
:1021700030BD4FF41651016000218180C180018182
:102180000C2242818181704710B5038A4FF2FF0211
:1021900013400A884C8822438C88C9880C43224308
:1021A0001A43028210BD0021018041808180C180DC
:1021B00070470029818902D041F4005101E021F4E7
:1021C00000518181704710B5C1F3421301F01F0423
:1021D0000121A140012B07D0022B07D01430002A87
:1021E000026805D00A4304E00C30F8E71030F6E747
:1021F0008A43026010BD002A828A01D00A4300E0AF
:102200008A4382827047028A22F00F020282028A87
:102210000A4302827047828922F4006282818289A5
:102220000A43828170470029818902D041F002016E
:1022300001E021F0020181817047028A22F0200230
:102240000282028A0A43028270470029018A02D070
:1022500041F4804101E021F4804101827047C1F3E3
:102260000801818070478088C0F308007047818929
:1022700041F0010181817047028BD2B20283028B4F
:1022800042EA012101837047028B02F47F420283FC
:10229000028B0A43028370470029818A02D041F0F1
:1022A000200101E021F02001818270470029818A0C
:1022B00002D041F0100101E021F01001818270474D
:1022C0000029818A02D041F0080101E021F00801D3
:1022D000818270470029818902D041F4004101E0E8
:1022E000C1F30E01818170470029818A02D041F437
:1022F000006101E021F4006181827047828A22F04E
:1023000004028282828A0A43828270470029818A7B
:1023100002D041F0020101E021F002018182704708
:102320000246002012880A4200D001207047C943AB
:102330000180704730B501F01F0201240025C1F370
:10234000421304FA02F2012B0FD0022B0FD0838A22
:102350004FEA11210088134204FA01F400EA040054
:1023600001D000B10125284630BD8389F0E7038AFA
:10237000EEE70A0A01219140C9430180704700003D
:10238000003801400044004000480040004C00403C
:10239000005000400CB500214B48019100910268AB
:1023A00042F4803202604FF4A063026802F400320B
:1023B0000092019A521C0192009A12B9019A9A4213
:1023C000F3D10268920333D5012100913F490A6895
:1023D00042F010020A600A6822F003020A600A68EA
:1023E00042F002020A604168416041684160416810
:1023F00041F480614160416821F47C114160416891
:1024000041F4E8114160016841F0807101600168A8
:102410008901FCD5416821F003014160416841F028
:10242000020141604168C1F381010229FAD10CBD6A
:1024300000910CBD244810B5016841F00101016014
:102440004168234A114041600168224A11400160FD
:10245000016821F480210160416821F4FE0141609E
:102460004FF41F018160FFF795FF1B494FF000609B
:10247000086010BD144910B54868184A10F00C03E4
:10248000174803D0042B01D0082B0AD002604968FA
:10249000134AC1F30311121D515C0268CA40026065
:1024A00010BD4A684B6802F470124FF0020413F436
:1024B000803F04EB924202D04B689B0301D5094B4D
:1024C00000E0064B5A43E1E70010024000200240C2
:1024D0000000FFF8FFFFF6FE08ED00E000127A00B2
:1024E0001400002000093D0024490A20087000F073
:1024F0007CFD02F073FA00F0B5FE00F03EFE01F044
:1025000023FD01F071FE00F015FA02F08FFB0120AF
:1025100000F044FA194C0125194E1A4FDFF8688073
:10252000DFF868B04EF6602A4FF00009A41C00BF27
:10253000C6F8A45102F097F90FF0D8FE02F02EF879
:10254000387808B100F0F1FED8F8000100282088A2
:102550000BD06428ECD3ABF8A09000F0D0FD0020A5
:1025600000F01CFAA4F80090E2E708B900F005FEBC
:1025700020885045DCD8401C2080D9E72800002066
:1025800000802142FA0000200000214200100020BB
:1025900042F6DF6303E01946491E89B2FCD2401EB1
:1025A00080B2F8D27047F0B5F549F64B01EB400226
:1025B00002F5905102F58052C3E90212B1F800C051
:1025C00000F5C06101F00706CD08F049EE4B0D445F
:1025D00017889C5D297867451CD2214200F5605020
:1025E000DFF8A8C300F007040CEBD00003D001789B
:1025F0001A5D11430CE0E64FBE5D31402970017851
:102600001B5D194205D00021118001783A5D11400F
:102610000170F0BD21432970F0BDF0B5D849D94C07
:1026200001EB400202F5905102F58052C4E902121A
:1026300000F5C062D54D02F0070705EBD203D44A7E
:102640001E78D75D3E401E7000F5B0531E4605EB68
:10265000D30306F007061F78965D00F560503740FB
:102660001F7005EBD00300F007001D78105C0540DB
:102670001D7000200880E1680880F0BDF0B5C04EF4
:10268000C24CC14DBF4B002006EB400101F59052FA
:1026900000F5B05701F58051BC46C3E9022104EBB7
:1026A000D7070CF0070C3F7815F80CC017EA0C0F91
:1026B00011D00F88128897420DD200F5C06C04EB40
:1026C000DC020CF0070C127815F80CC012EA0C0FA3
:1026D00001D17F1C0F80401C80B2C828D4D3F0BD2C
:1026E000F0B5A74EA94CA84DA64BC82006EB40015B
:1026F00001F5905200F5B05701F58051BC46C3E991
:10270000022104EBD7070CF0070C3F7815F80CC03A
:1027100017EA0C0F11D00F88128897420DD200F5DE
:10272000C06C04EBDC020CF0070C127815F80CC03E
:1027300012EA0C0F01D17F1C0F80401C80B2F628DA
:10274000D4D3F0BDF0B58E4E904C8F4D8D4BF6200E
:1027500006EB400101F5905200F5B05701F58051AC
:10276000BC46C3E9022104EBD7070CF0070C3F7805
:1027700015F80CC017EA0C0F11D00F881288974279
:102780000DD200F5C06C04EBDC020CF0070C1278E3
:1027900015F80CC012EA0C0F01D17F1C0F80401CF1
:1027A00080B2FA28D4D3F0BDF0B5754E774C764D93
:1027B000744BFA2006EB400101F5905200F5B0573A
:1027C00001F58051BC46C3E9022104EBD7070CF0A8
:1027D000070C3F7815F80CC017EA0C0F11D00F88C2
:1027E000128897420DD200F5C06C04EBDC020CF0AD
:1027F000070C127815F80CC012EA0C0F01D17F1CDF
:102800000F80401C80B2FF28D4D9F0BD2DE9F047DD
:102810004FF08040002606825A4DA8880A30A880D2
:102820002878401C287000F021FA2878574C564F21
:10283000632808D92E7094F8E1013979084384F8A7
:10284000E101FFF77FFF29784FF00A09B1FBF9F2A8
:10285000A84609FB12104E4D072807D1FFF740FF8D
:1028600094F8E101E978084084F8E10198F8001053
:10287000B1FBF9F309FB1312022A05D194F8E12107
:10288000FB781A4384F8E121322907D1FFF7F6FEDD
:1028900094F8E1012979084084F8E10198F80000F2
:1028A0005A280AD1FFF780FFB8F802103948491CAE
:1028B000A8F8021006703848067098F8000000F07A
:1028C0000F00022803D102F018F902F0B6F9B8F8A7
:1028D00002004A46B0FBF2F309FB1303052B07D1B4
:1028E00094F8E13195F805C003EA0C0384F8E1316E
:1028F000B0FBF2F309FB13022AB994F8E1217B79CA
:102900001A4384F8E121B0F5967F07D058B1B0F5AD
:10291000167F01D3A8F80260BDE8F08794F8E101C2
:10292000A979084003E094F8E101B979084384F8F3
:10293000E101F1E73EB501210846FEF74FFD48F6FB
:10294000A040ADF804000120ADF800000020ADF873
:102950000600ADF802004FF0804469462046FEF7BD
:10296000A3FE01212046FFF77EFB012211462046EF
:10297000FFF758F901212046FFF73FF93EBD00005F
:1029800000100020E0000020EC5F00080010002094
:10299000F45F00080C0100200D0100202DE9F84330
:1029A000054600214FF00060FDF75CFC4FF48060AD
:1029B000FDF724FC25208DF8000002268DF801602B
:1029C00000248DF802408DF803506846FDF71BFC8B
:1029D0000E208DF800004FF003088DF801808DF86F
:1029E000026001268DF803606846FDF70CFC272085
:1029F0008DF800008DF801608DF802408DF80350CD
:102A00006846FDF700FC1D208DF8000005208DF8BC
:102A100001008DF802408DF803506846FDF7F3FB86
:102A20001E208DF8000004278DF801708DF80240FB
:102A30008DF803506846FDF7E6FB32208DF8000064
:102A400006208DF801008DF802408DF8035068468D
:102A5000FDF7D9FB2E208DF800008DF801408DF890
:102A600002608DF803606846FDF7CDFB1C208DF8F1
:102A700000008DF801408DF802408DF80350684643
:102A8000FDF7C1FB28208DF800008DF801708DF84E
:102A900002408DF803506846FDF7B5FB17208DF80E
:102AA00000008DF801808DF802408DF803506846D3
:102AB000FDF7A9FBBDE8F8831CB50F210020FEF748
:102AC000FCFA4FF48050009000208DF804000C2098
:102AD0008DF8050001208DF806006846FDF73AFFE5
:102AE0004FF4006000906846FDF734FF1CBD1CB534
:102AF00009210220FEF7E1FA4FF400700090002057
:102B00008DF804000C208DF8050001208DF80600DA
:102B10006846FDF71FFF08210220FEF7CEFA4FF4AA
:102B2000807000906846FDF715FF07210220FEF730
:102B3000C4FA802000906846FDF70CFF06210220B1
:102B4000FEF7BBFA402000906846FDF703FF1CBD6E
:102B500038B50120ADF8000004258DF8035002249B
:102B60008DF802406946FE48FEF7EFF92003ADF804
:102B700000008DF80350FB4D8DF802406946284651
:102B8000FEF7E3F94FF44070ADF8000014208DF823
:102B900003008DF802406946F348FEF7D6F94FF47A
:102BA000E070ADF8000010208DF8030003208DF8D0
:102BB000020069462846FEF7C8F938BD38B5CE2070
:102BC000ADF8000004248DF8034002258DF8025072
:102BD0006946E348FEF7B9F94FF20300ADF800008B
:102BE0008DF803408DF802506946DF48FEF7ADF9D5
:102BF0003020ADF800008DF803408DF80250694692
:102C0000D848FEF7A2F938BD38B54FF41940ADF8F1
:102C1000000001248DF8024010258DF8035069460C
:102C2000CF48FEF792F9F820ADF800008DF8024089
:102C30008DF803506946CC48FEF787F94FF4F05001
:102C4000ADF800008DF802408DF803506946C54884
:102C5000FEF77BF90420ADF800008DF802408DF8F6
:102C600003506946C148FEF770F938BDF0B5C04C55
:102C7000D4F80451BF48C14900220378BE4890F8F7
:102C800080601DB10A7026F0010508E091F900503E
:102C90009D4202DA6D1C0D7003E046F0010580F8DC
:102CA0008050D4F808512DB14A7090F8805025F02A
:102CB00002050AE091F901509D4202DA6D1C4D7047
:102CC00005E090F8805045F0020580F88050D4F877
:102CD0000C512DB18A7090F8805025F004050AE05F
:102CE00091F902509D4202DA6D1C8D7005E090F85A
:102CF000805045F0040580F88050D4F818512DB16B
:102D0000CA7090F8805025F008050AE091F9035048
:102D10009D4202DA6D1CCD7005E090F8805045F0C0
:102D2000080580F88050D4F81C412CB10A7190F845
:102D3000804024F010040AE091F904409C4202DA39
:102D4000641C0C7105E090F8804044F0100480F899
:102D500080408B4DD5F810412CB14A7190F88040DD
:102D600024F020040AE091F905409C4202DA641C38
:102D70004C7105E090F8804044F0200480F88040D9
:102D8000D5F814412CB18A7190F8804024F04004A9
:102D90000AE091F906409C4202DA641C8C7105E05D
:102DA00090F8804044F0400480F88040754CD4F89E
:102DB00000512DB1CA7190F8803023F080030AE0F1
:102DC00091F907509D4202DA6D1CCD7105E090F833
:102DD000803043F0800380F88030D4F80471664D71
:102DE000B5F8283E95F881601FB10A7226F00105FA
:102DF00008E091F908509D4202DA6D1C0D7203E063
:102E000046F0010580F88150D4F830512DB14A7256
:102E100090F8815025F002050AE091F909509D4291
:102E200002DA6D1C4D7205E090F8815045F0020504
:102E300080F88150D4F834512DB18A7290F88150C5
:102E400025F004050AE091F90A509D4202DA6D1C52
:102E50008D7205E090F8815045F0040580F88150AE
:102E6000D4F838512DB1CA7290F8815025F0080578
:102E70000AE091F90B509D4202DA6D1CCD7205E01B
:102E800090F8815045F0080580F88150D4F83C5105
:102E90002DB10A7390F8815025F010050AE091F9E0
:102EA0000C509D4202DA6D1C0D7305E090F88150C4
:102EB00045F0100580F88150D4F81C512DB14A73AB
:102EC00090F8815025F020050AE091F90D509D42BF
:102ED00002DA6D1C4D7305E090F8815045F0200535
:102EE00080F88150D4F820512DB18A7390F8815028
:102EF00025F040050AE091F90E509D4202DA6D1C62
:102F00008D7305E090F8815045F0400580F88150C0
:102F1000D4F824412CB1CA7310F8811F21F080012C
:102F20000AE091F90F209A4202DA521CCA73F0BDEE
:102F300010F8811F41F080010170F0BD0E4B10B5FB
:102F400013F8A00F0E4900F00102C1F8A421084AAD
:102F5000C0F34004C2F8A041C0F3800414E00000B4
:102F60000008014000100140000C01400014014025
:102F700000002142F000002000100020AC070020DB
:102F80000000224200802142C2F8AC41C0F3C004DC
:102F9000C2F8B041C0F30014C2F8BC41C0F3401203
:102FA000C1F8A821C0F38012C1F8AC21C009C1F852
:102FB000B0015878184A00F00101C2F88811174989
:102FC000C0F34002C1F88C21C0F38002C1F8902107
:102FD000C0F3C002C1F89421C0F30012C1F89821D7
:102FE000C0F34010C1F89C0110BD10B501213C2078
:102FF000FEF7EBF901210846FEF7E7F90749012042
:10300000C1F8A401FFF700FEFFF798FFFFF7D6FD18
:10301000BDE810409CE50000008022420080214273
:1030200010B50E48002404800D48D0F824210D4925
:10303000C0F8A44122B1B1F8180F401CA1F8180F34
:1030400091F8F201800707D50448002201211038C9
:10305000FEF7E8FD0448047010BD000010040040B5
:103060000000224200100020F100002038B1774912
:10307000774B91F8E721DB791A4381F8E72175490D
:10308000A1F87E0E70472DE9F04105460C281BD2B1
:10309000FDF7DFFC704E06EBC520FDF715FD0024A3
:1030A0006E4FED024FF4806805EB4400304480B26F
:1030B00037F81410FDF7CBFD641CA4B24445F3D3DC
:1030C000BDE8F041FDF7D1BCBDE8F08170B50C283A
:1030D00014D20021C3026248604C4FF4806500BFE7
:1030E00003EB410292B2865C0244527806EB022264
:1030F00024F81120491C89B2A942F1D370BD30B423
:10310000544A5649002041F2F41341F2B63400BF4C
:1031100032F8135021F81050401C5B1C9BB280B257
:10312000A342F5D340F2645340F2965432F8135060
:1031300021F81050401C5B1C9BB280B2A342F5D317
:1031400040F6640340F6960432F8135021F810500C
:10315000401C5B1C9BB280B2A342F5D35FF02003FE
:1031600032F8134021F81040401C5B1C9BB280B227
:10317000402BF5D330BC0A2085E730B500240A2067
:10318000FFF7A4FF3548334941F2F41241F2B63358
:1031900030F8145021F81250641C521C92B2A4B2A0
:1031A0009A42F5D340F2645240F2965330F81450EC
:1031B00021F81250641C521C92B2A4B29A42F5D368
:1031C00040F6640240F6960330F8145021F812508D
:1031D000641C521C92B2A4B29A42F5D35FF0200252
:1031E00030F8143021F81230641C521C92B2A4B290
:1031F000402AF5D330BD17494FF480524FF43D5368
:10320000002000BF21F81200521C92B29A42F9D35A
:103210004FF4A0624FF4C06321F81200521C92B226
:103220009A42F9D34FF400624FF4106321F8120070
:10323000521C92B29A42F9D35FF0000221F81200B8
:10324000521C92B2802AF9D370470000001000206F
:10325000EC5F00080010002000600008886E00206D
:103260000060000830B5F9485221F94B8181F94AD4
:10327000002000BF33F8105000F5E064401C80B21D
:1032800022F814507E28F5D3F34B4FF6FF74F34A1F
:10329000585C194404EA002049780843F04910803A
:1032A000092081F8E001E949C82010310870487010
:1032B00030BD2DE9F0410546112821D2FDF7C9FBAB
:1032C000E84E06EBC520FDF7FFFB0024EF02E64DBC
:1032D0004FF4806805EB840235F82410927807EBF0
:1032E0004400304401EB022180B289B2FDF7AFFC0B
:1032F000641CA4B24445EDD3BDE8F041FDF7B5BB75
:10330000BDE8F08130B511280ED2D34CD64B002148
:103310004FF4006501EBC02292B2A25C23F81120A9
:10332000491C89B2A942F5D330BDC84801780029AB
:1033300009D00021017081714189CC488164416CC0
:1033400041F001014164704770B50024012805D0A7
:10335000C34902282BD0032833D038E00020FFF7E0
:10336000D1FFC1490F204FF6FF72A1F8B800A1F8B4
:10337000BA405E204FF4006321F81020401C80B258
:103380009842F9D3FDF765FBB948FDF79DFB002096
:10339000FFF78FFFB34D012405EBC420FDF794FB2D
:1033A000641CA4B20A2CF7D3FDF75FFB0FE04FF4C7
:1033B000005047F67E624454801C80B29042FAD39B
:1033C00005E000204454801C80B2BE28FAD3A949ED
:1033D000062048709D490120488170BD9B4A10B568
:1033E000128900230321C01C521E05E010F8014B76
:1033F000491C2344DBB289B29142F7DB184610BD69
:10340000F0B5924904209C4C09899C4A994D891E2B
:103410000BE02718235C7F7805EB5006D35CD75D63
:10342000801C07EB0313337080B28842F1DBF0BDE0
:103430009048C178807800EB0120844988817047EA
:103440008C48C178007900EB01208049C881704721
:10345000F8B57F49DFF8F4C1002231F81000009080
:1034600084490220854B487010469CF80540143B67
:10347000EE4610E01EF8007001EB400603EB171556
:1034800007F00F072D78B570DF5D401C3D442A44DE
:10349000F770D2B280B2A042ECD301EB400103241A
:1034A000D21C8C70D2B203EB121402F00F022478FB
:1034B000CC709A5C0A71042101EB4000ACF80A0060
:1034C000F8BDA0F58041B1F57A5F02D2A0F50050B9
:1034D00032E0A0F520717C2917D94031A0F5E072C7
:1034E000162901D890B27047A0F5C073162B01D8E9
:1034F000E03821E0A0F500731F2B02D8A0F5A070E2
:103500001AE0A0F5A0631F2B01D888B27047A0F580
:10351000F0711F2901D820380EE0BF2802D800F52D
:10352000807009E0A0F1C001BF2902D800F58860D1
:1035300002E01F2AEAD8203080B270474FF4C06200
:10354000904202D200F5006034E0A0F5C0619142E3
:1035500002D200F508502DE0A0F54061B72902D84D
:10356000A0F5E06026E0A0F59052A0F56061BF2ACA
:1035700001D888B27047A0F5A053B3F57A7F01D285
:1035800098B27047A0F52053FF2B01D890B2704736
:10359000A0F58052FF2A02D8A0F520600AE0FF299A
:1035A00002D800F5807005E0A0F57061FF29EED823
:1035B000A0F5807080B270472DE9F04302202D4EB7
:1035C000DFF8B880002770703C46A8F114081F4D42
:1035D00023E0A889204480B2FFF773FFDFF88090D2
:1035E00006EB440C10F8091008EB111000788CF869
:1035F0000200A889204480B2FFF763FF10F8090099
:10360000641C00F00F01A4B218F801008CF803004C
:103610009CF8021008443844C7B268798442D8D371
:1036200006EB440003218170FF1CF9B208EB111373
:1036300001F00F011B78C37018F80110017104200C
:1036400000EB44006881BDE8F0830000F400002036
:10365000863E010800100020006000080050002095
:103660000010002000600008886E0020000002406A
:10367000006800088C7E0020808000209A400108AD
:10368000F0B5F94E0422F94DB178F07802EB012142
:103690000844A8810024F64F09E0A889204480B29C
:1036A000FFF70FFF3119641C4979C155A4B268793D
:1036B0008442F2D30620707001206881F0BD30B5DD
:1036C000E94CE078A17800EB012080B2FFF736FFEB
:1036D000E74901EBD005E078A17800EB012080B24A
:1036E000FFF72CFFE34900F00700085C2978084346
:1036F00028700620DD4960700120488130BD30B55A
:10370000D94CE078A17800EB012080B2FFF716FFDA
:10371000D74901EBD005E078A17800EB012080B219
:10372000FFF70CFFD44900F00700085C2978084037
:1037300028700620CD4960700120488130BDCA48FC
:10374000C178807801EB0020C84980B28881A0F55B
:103750006060023804D0C82800D02DE7652000E062
:10376000012075E630B5C14CA089A0F56062233A0E
:1037700015D00921BE4D012A17D0022A1AD085F88A
:10378000E011FFF7DBFE05EBD005A089FFF7D6FEC1
:10379000B84900F00700085C297808432870B2494E
:1037A000062048700120608130BD85F8E0110020BE
:1037B0006070F4E70A2085F8E001F0E730B5AB4C23
:1037C000A089FFF7BBFEAA4901EBD005A089FFF74E
:1037D000B5FEA94900F00700085C29780840A24915
:1037E0002870062048700120608130BD2DE9F04F1F
:1037F000DFF874A2022100248AF801109AF804105C
:103800009AF8030001EB002080B2FFF75AFEDFF8C0
:103810005CB241F290718842ABF80C0003D0A0F585
:10382000B852D03A5CD188425AD1DFF85082002594
:103830002F4698F800C4A8F5805924E009EB47000A
:1038400000F580504E46B0F80404FFF73AFE06EB50
:103850004502400802F5805236F81010A2F8901781
:103860006D1CA0F5C061ADB26E290AD806EB400010
:10387000418806EB450000F580506D1CA0F89017BC
:10388000ADB27F1CFFB26745D8D398F802C40026BA
:1038900024E0B91909EB410000F58050C846B0F8A2
:1038A0000404FFF74BFE020938F8121000F00F0273
:1038B000012000FA02F38B4305EB161208EB4201DC
:1038C00001F5805106F00F03B1F8902700FA03F0DC
:1038D00010D08243761CA1F89027F6B26645D8D363
:1038E0000020BBF80C809BF8056065495346DFF863
:1038F000809116E00243EDE708EB000703EB400C74
:1039000017F80950401C01EB151705F00F053F781B
:103910008CF802704D5D8CF803503D442C44E4B2A9
:1039200080B2B042E8D30AEB40030325E41C9D704B
:10393000E4B201EB141504F00F042D78DD70095D7D
:103940001971042101EB4000ABF80A00BDE8F08FCB
:10395000F0B5454E454D00243079F178444F00EBE9
:103960000120A88109E0A889204480B2FFF7A9FDC1
:103970003119641C8979C155A4B268798442F2D3A3
:103980000620707001206881F0BD2DE9F043364AB1
:10399000364C02205070E0890023A0F5004085B22B
:1039A000E581184666793649DFF8D89016E000BF01
:1039B00005EB000C19F80C8002EB400C01EB18171A
:1039C00008F00F083F788CF8027011F80880401C4E
:1039D00047443B448CF80380DBB280B2B042E7D36B
:1039E00002EB40020325DB1C9570DBB201EB1315E3
:1039F00003F00F032D78D570C95C1171042101EB20
:103A0000400060811FE62DE9F047174E174CDFF8A4
:103A100060C03079F178012700EB012080B20A21E3
:103A2000A0818CF8E0116770B0F5004F49D3164AB9
:103A30000021A0F500401170A0810D4604F110088E
:103A4000DFF8489039E0A0894319DA0A88F80020A5
:103A500098F8010082421BD17019514203EBC12238
:103A6000807929F8120026E08C7E0020F4000020E6
:103A700000100020EC5F0008F45F00080020002028
:103A800086400108006000083B000020886E00208E
:103A9000FFF70FFC98F80000FFF734FC98F80000DF
:103AA00088F80100A28971192A44404202EBC02221
:103AB000897929F812106D1CADB260798542C2D3A4
:103AC00011E0001DA08100250AE0A089284480B2F1
:103AD000FFF7F7FC71196D1C897900F80C10ADB275
:103AE00060798542F1D3062070706781BDE8F08768
:103AF00070B505230A0ACCB2A0F50040F74980B2A0
:103B000045F6DB650E5CA64203D10E187678964228
:103B100005D0801C80B2A84201D8032BF2D800F552
:103B2000004080B270BD2DE9F041ED4CED4D607963
:103B3000A17900EB012081B2E889FFF7D9FFE88184
:103B400002216170020AC3B23121E748A17000EB83
:103B5000121102F00F020978E170865C00EB13127B
:103B60002671127803F00F036271C35C3131314466
:103B700011441944C91CC9B2A371032700EB1112E7
:103B8000E771127801F00F012272405C6072092027
:103B90006881BDE8F08130B50A280FD2D34CD44BF0
:103BA00000214FF4006500BF01EBC02292B2A25C7D
:103BB00023F81120491C89B2A942F5D330BD2DE963
:103BC000F84FC84F05468946B97000F5004080B2ED
:103BD0000F21FFF78DFF4844A0F5004084B25B2D14
:103BE0002BD9A5F15C0001040E0DB978A4F15C009D
:103BF0004908C0F34E00C00801F00702CB08BA70B4
:103C0000BC490EE00F1811F800C017F8017C07EB53
:103C10000C2797403F0A00EB030C401E01F80C7084
:103C200080B2B042EED10E180F5C16F8016C184449
:103C300006EB07269640320A0A544FEAD42AE00AD5
:103C40000090B0EBD52F02D1C5F30A0600E00026A4
:103C5000BAEBD42F03D1C4F30A077F1C01E04FF461
:103C600000670098FFF74EFBE20AD2023046DFF809
:103C70007CB2DFF87CC27B1C0BE000BF02EB0008CB
:103C8000A8EB090189B21BF801102CF81010401C98
:103C900080B29842F2D30098FFF70BFBB81B201AB2
:103CA00084B205EB0900A042C9D3BDE8F88F2DE925
:103CB000F0418B4F8B4D7879B979081A10F0FF01DC
:103CC00005D0E889A0F5004080B2FFF778FF8A4967
:103CD0000020844C0870642010344FF4004220709F
:103CE0006070F978387902EB01210844A881B8792D
:103CF00068710026DFF8F88120E0A8898219D10ACE
:103D000021706078814207D1B819C379484202EB2B
:103D1000C02128F811300FE0FFF7CBFA2078FFF729
:103D2000F1FA20786070AA89B9193244404202EB56
:103D3000C022C97928F81210761CB6B2687986427A
:103D4000DBD32078FFF7B5FA062078700120688170
:103D50001FE76448C8211030417001706049062097
:103D60004870604901204881704710B55D4C10349F
:103D70006078FFF79EFAC82060702070FCF775FE2F
:103D800057490620487057490120488110BD70B539
:103D9000544A10890B2805D158480379372B11D084
:103DA000382B0FD0FFF74CFB4D49887861284BD05A
:103DB00026DC11283FD01EDC98B3012838D010280B
:103DC0002AD132E048498479143145790C5D4D5D42
:103DD00004EB0514C579007A4D5D085C2D0305EBF5
:103DE000002020449081372B02D0BDE87040E5E4EC
:103DF000BDE87040B6E4412823D060280CD126E00D
:103E0000772821D004DC622825D0632804D120E063
:103E1000872813D0D12823D0152048700120508145
:103E200070BDFFE7BDE87040E0E4BDE870408FE59D
:103E3000BDE87040A9E5BDE87040E4E5BDE870402C
:103E400093E7BDE870406EE6BDE8704081E7012071
:103E500002E0022000E00320BDE87040FFF774BAE2
:103E6000BDE8704023E71F4810B51D4906230489AB
:103E700001224B70428110BD70B5FFF7C1FA1F4897
:103E8000174D184CC07837281BD006DC30280BD0D3
:103E900031280ED0342837D110E0382816D04228E7
:103EA00019D0452830D12BE028796071FFF747FC05
:103EB0002AE028796071FFF7E3FB25E0FFF7D3FFE5
:103EC00022E0FFF7B5FAFFF7FAFB1DE0FFF7B0FAC3
:103ED000FFF715FC18E0FFF748FF15E00060000849
:103EE0008C7E0020F400002086400108005000086D
:103EF000886E002000D200203B000020808000203F
:103F000068796071FFF743FF6189208901434FF0B1
:103F1000010002D115216970608100212181A07109
:103F20007EE71FB5694600900020ADF80400ADF8AB
:103F30000600ADF80800ADF80C000C20ADF80A0042
:103F40008F48FEF7C3F81FBD10B501218CB0880360
:103F5000FDF73BFA01210846FDF72EFA894C204671
:103F6000FCF706FC86480021001D00908648019061
:103F7000102002908F20CDE903018020CDE90501BA
:103F80008001CDE9081007910A9169462046FCF7A7
:103F90005CFC012202212046FCF78CFC4FF4964089
:103FA000FFF7BFFF764C012240F225512046FEF775
:103FB0000AF9012280212046FEF71DF90121204641
:103FC000FEF7F7F86015ADF82C0003208DF82E00F1
:103FD00018206E4C8DF82F000BA92046FCF7B5FF7A
:103FE0002015ADF82C0004208DF82F000BA92046D9
:103FF000FCF7ABFF0CB010BD62484438416841F497
:1040000000514160416C4FF6FE72114041646049BD
:104010000120087070472DE9F0475948001D0088BD
:10402000DFF8709100F07F0000250126584C89F8D8
:1040300000004FF00608A9F5FA77052804D00228F9
:1040400009D0208948B11BE0258187F8018066816D
:10405000FFF76BF911E0268112E0207901281ED0CC
:1040600000281BD14FF41650FFF75BFF258187F81E
:1040700001806681FFF759F92671208900280DD04B
:104080002089CC46401C80B2208199F8001009F8A4
:104090000010B0F5C87F0ED96581258126E54FF463
:1040A0009640FFF73EFF258187F801806681FFF784
:1040B0003CF92571E1E70328F0D9604410F8020CBF
:1040C0000328EBD13348FFF789F9E07021890CEB25
:1040D000010212F8013C304A02EB10152D78AB4278
:1040E00009D100F00F001CF80110105C814202D1D0
:1040F000BDE8F047C0E6152078706681BDE8F0475E
:10410000FFF713B970B51E4C40F2255529462046DD
:10411000FEF710F9012805D129462046FEF729F9B6
:10412000FFF779FF08212046FEF7FAF8012806D1AB
:1041300008212046FEF7FBF82046FEF794F840F2EF
:10414000277529462046FEF7F5F8012808D12946AB
:104150002046FEF70EF9002229462046FEF733F8E6
:1041600040F2266529462046FEF7E4F8012805D1ED
:1041700029462046BDE87040FEF7FBB850E6000037
:1041800000380140440002408D7E002000080140BC
:10419000F4000020808000208640010870B5F94DB1
:1041A000FF22134605F5807606E000BF10F8014BAC
:1041B00054402A5D5A40335D491EF7D243EA02203B
:1041C00070BD1FB5694600900020ADF80400ADF841
:1041D0000600ADF80800ADF80C000C20ADF80A00A0
:1041E000E948FDF773FF1FBD38B501218804FDF7CD
:1041F000F5F801210820FDF7E8F84FF40060ADF86C
:1042000000000420E14C8DF8030069462046FCF7CD
:104210009CFE2015ADF8000003208DF80200182048
:104220008DF8030069462046FCF78FFE4FF4964058
:10423000FFF7C7FFD44C012240F225512046FDF77D
:10424000C2FF01212046FDF7B4FFD1480021A0F8AC
:10425000041F0121A0F8F21E38BD2DE9F04FCD4E0C
:10426000CD4C314696F801C0887891F803804A79A0
:104270000B798146C64908EB0020002589B041F240
:104280006F7B4FF4FA5E01EB4001A6F16407BCF1CD
:10429000050F6FD018DCBF4BEA46BCF1010F1B784D
:1042A0006BD0BCF1020F67D0BCF1030F02D0BCF1A0
:1042B000040F5CD18DF8003051008DF801C08146AB
:1042C0008DF802100020E3E0B24A4FF6FF79BCF10E
:1042D000060F9378D27802EB0322AD4B03EB420238
:1042E00002F500527CD0BCF10F0F40D0BCF1100F92
:1042F0003DD1DFF8A0C258459CF807309CF808C0B3
:1043000004D809EA0328E044A2F80080704508D3E5
:10431000A1F58051138091F8601009EA01206044F2
:1043200010806570A5710020A179325C401C7A5420
:10433000491CC0B2A1710628F6D306219548FFF7A3
:104340002DFFA060A179020A7A54491CC9B201224A
:104350007854491CA17140F227718B48FDF733FF57
:1043600000203554401CC0B20A28FAD9E57009B0C3
:10437000BDE8F08FE8E000E033E08DF800308DF824
:1043800001C08DF802908DF80380B1F8A000010AF9
:104390008DF804108DF8050006215046FFF7FEFE4B
:1043A000010AA0608DF806108DF807006570A571F0
:1043B00000205246A179135C401C7B54491CC0B2BA
:1043C000A1710728F6D9012240F227716E48FDF746
:1043D000FAFE00203554401CC0B20A28FAD9C5E7BD
:1043E00089E08DF800308DF801C08DF802908DF8CD
:1043F0000380B1F88000010A8DF804108DF80500E3
:1044000006215046FFF7CAFE010AA0608DF806108B
:104410008DF807006570A57100205246A179135CE4
:10442000401C7B54491CC0B2A1710728F6D9012257
:1044300040F227715448FDF7C6FE00203554401C59
:10444000C0B20A28FAD991E709EB000159450DD805
:104450004F4B0AEB400C03EB400303F500531B8862
:104460004FEA13288CF803808CF8043071450DD383
:10447000474B03EB4101A1F580510AEB4003B1F832
:1044800060104FEA112C83F803C01971401CC0B2B0
:104490008242D9D89DF802105046C91CFFF77EFE13
:1044A000A0609DF802300DF10301020A5A549DF8F4
:1044B000022001A9D44650546570A5719DF80210E0
:1044C0000020091D08E000BFA2791CF80030BB5491
:1044D000521C401CA271C0B28142F5D2012240F2AE
:1044E00027712948FDF76FFE00203554401CC0B2EB
:1044F0000A28FAD93AE727494FF6FF78584591F844
:1045000004C0497908EA0C2C614489B200D81180B2
:10451000704500D311806570A5710020A179325CCF
:10452000401C7A54491CC0B2A1710728F6D9012257
:1045300040F227711448FDF746FE00203554401C18
:10454000C0B20A28FAD911E702EB0320A1F8A000B3
:104550006570A5710020A179325C401C7A54491C19
:10456000C0B2A1710728F6D9012240F2277106488E
:10457000FDF729FE00203554401CC0B20A28FAD9A4
:10458000F4E60000E740010800480040000C01404C
:1045900000100020D8820020080100202DE9F04101
:1045A000604C2079002854D12078002601284DD174
:1045B0005D4F2670B7F8040FF0BB5C4DB7F8F21EE4
:1045C0002878884242D1A07808280AD909212846AB
:1045D000FFF7E4FDA060AA7AC1B2914210D1697AD6
:1045E00009E006215148FFF7D9FDA060EA79C1B280
:1045F000914205D1A979B1EB102F01D1FFF72DFE22
:10460000B7F8040F012821D12878B7F8F41E8842A2
:104610001CD105214548FFF7C1FDA060AA79C1B2B0
:10462000914213D16979B1EB102F0FD12879E97834
:1046300000EB01203E4900E008E0A1F89C000020CA
:104640002E54401CC0B20A28FAD9A670A6700120C8
:104650002071BDE8F0812DE9F041364D40F225563C
:1046600031462846FDF766FE2E4C08B331462846F3
:10467000FDF77FFE2079D8B12846FDF7F4FD61797A
:104680002A4EC0B2012709B93070677126493078C7
:10469000B1F8F21E88420BD12846FDF7E4FD014631
:1046A000A0783154401CC0B2A070072800D32770F6
:1046B00008212846FDF734FE012806D108212846A6
:1046C000FDF735FE2846FDF7CEFD40F22776314650
:1046D0002846FDF72FFE012815D11449607864396A
:1046E000095C401C60702846FDF7B9FD6078A1792F
:1046F000884204D1002231462846FDF764FD314648
:104700002846FDF736FE40F2266421462846FDF78E
:1047100011FE01289DD121462846BDE8F041FDF754
:1047200028BE96E70801002000100020D882002053
:10473000003000200048004081070CD16421B0FB0C
:10474000F1F201FB120141B94FF4C871B0FBF1F273
:1047500001FB120008B100207047012070472DE9CD
:10476000F05F99460546DDE90AAB0023A0F5FC6041
:1047700090460E46792802D30120BDE8F09F4FF401
:10478000FC64B34FDFF8CCC208E02046FFF7D4FF4B
:1047900008B13B4400E06344641CA4B2AC42F4D3CF
:1047A000761EF6B20024AC4FDFF8B0C20EE0385DE2
:1047B00040F2A321484303EBC0132846FFF7BCFF98
:1047C00010B1012C00D16344641CA4B2B442EED3F6
:1047D00040F2A32108FB01F0A04903EBC0104942BD
:1047E0000844C9EB4912C2EB092100EB0110CAEBE6
:1047F0000A1100EB810000EB0B040120FCF790FC98
:10480000FCF784FE2046FCF74FFEFCF77FFE0020FD
:10481000B3E730B54FF4C87303290FD2840706D12C
:104820004FF47A74B0FBF4F504FB150424B9B0FB23
:10483000F3F403FB14040CB9521ED2B2B0FBF3F331
:10484000024402EB90021A446423B0FBF3F0101A06
:10485000834A801E515C0844072190FBF1F201FB62
:104860001200C0B230BD2DE9FC417E487E497F4C2C
:1048700090F8E121CB791A4211D094F81A0E94F8ED
:104880001C1ECDE9001094F81E3E94F8202E94F8DA
:10489000221EB4F8240EFFF762FFBDE8FC8190F8F9
:1048A000E20189780842F8D0FCF7F5FDDFF8ACC1E9
:1048B0000646B0FBFCF36A48801E0188994234D05A
:1048C00003804FF4FC654FF4B7784FF4B6770FE0F0
:1048D0002846FFF731FF38B1434502D3A3F5B7733C
:1048E00004E06D1CADB205E0A3F26D136D1CADB21A
:1048F000BB42EDD8A4F8245E0025574F0DE000BF61
:10490000B4F8220EFFF718FF08B1012D36D0785DFC
:10491000984204D81B1A6D1CADB21C2BF0D26D1C32
:10492000A4F8225E5B1CA4F8203EB6FBFCF00CFB56
:1049300010604FF46161B0FBF1F2A4F81E2EB0FBE1
:10494000F1F201FB12033C22B3FBF2F3A4F81C3E8C
:10495000B0FBF1F301FB1300B0FBF2F102FB11001D
:10496000A4F81A0E94F8202E94F8221EB4F8240EFF
:1049700004F61A64FFF74DFFA0818EE71D2BCED3FE
:104980001D3BC8E710B501214FF0C050FCF726FDD4
:104990000120FCF7C5FBFBF721FE0120FCF7B2FC70
:1049A0004120FCF738FC0028FAD04FF48070FCF767
:1049B000BAFC0120FCF7BCFCFCF7AEFDFCF7A6FD41
:1049C00001210846FCF750FDFCF7A0FD47F6FF70FB
:1049D000FCF777FDBDE81040FCF798BD10B504204A
:1049E000FBF725FE45F65A24A04206D0FFF7CAFF82
:1049F00021460420FBF714FE1AE001214FF0C050BD
:104A0000FCF7ECFC002041F28831401C80B2884267
:104A1000FBD37B20FCF7FFFB10B97A20FCF7FBFBF4
:104A2000FCF701FD01210846FCF71EFDFCF76EFDB9
:104A30000C480D4A90F8E211927811430C4A80F824
:104A4000E21190F8E111D279114080F8E11110BD26
:104A50000085E2018033E101E74201088051010055
:104A60001601002000100020EC5F0008001000205C
:104A7000F45F000810B586B001210420FCF7A5FC06
:104A800001214807FCF7AAFC3020ADF810000024F3
:104A90008DF8134004A92448FCF757FA3C20CDE9CF
:104AA00000040220039069460020FBF7EFFD6946F1
:104AB0001020FBF7EBFD01210020FBF7FFFD01219A
:104AC0001020FBF7FBFD01210020FBF70BFE01216D
:104AD0001020FBF707FE00210846FBF725FE00210A
:104AE0000846FBF728FE01210020FBF7FBFD012112
:104AF0001020FBF7F7FD06B010BD10B50B4C0020E1
:104B0000B4F8A01EFBF710FEB4F8A21E0020FBF7BD
:104B100012FE01210020FBF7E5FD0121BDE8104058
:104B20001020FBF7DFBD000000080140001000204E
:104B300030B591B001214FF40470FCF746FC01211F
:104B40000846FCF739FC0F20ADF8400000248DF832
:104B5000434010A94848FCF7F8F9484D2846FBF7B0
:104B600007FE474800904748CDE901044FF4C8705C
:104B7000CDE9030480200590400006908000079056
:104B8000202008900002CDE9090469462846FBF779
:104B90005CFE01212846FBF782FE01208DF83000E3
:104BA0008DF831000B944FF46020CDE90D04344CA6
:104BB00004208DF83C004C3C0BA92046FBF792FBEF
:104BC000072301220A212046FBF70CFC07230222BF
:104BD0000B212046FBF706FC072303220C2120466D
:104BE000FBF700FC072304220D212046FBF7FAFB0C
:104BF00001212046FBF7A8FB01212046FBF79AFB89
:104C00002046FBF7B4FB2046FBF7B6FB0028FAD1A1
:104C10002046FBF7B8FB2046FBF7BAFB0028FAD189
:104C200001212046FBF7BBFB11B030BD10B5FFF7EB
:104C30007FFFBDE81040FFF71DBF70B50022114B8C
:104C4000114D10466424002103EBC10636F81060B4
:104C5000491CC9B232446429F6D392FBF4F105EB46
:104C6000400202F58042401CA2F81C1F0022C0B284
:104C70000428E8D370BD0000001001400800024085
:104C80004C2401403C8300200010002053EA020C19
:104C900000F069802DE9F04B4FF00006002B1FBF9C
:104CA000B3FA83F503FA05F424FA05F65E4012BF61
:104CB0001643B2FA82F502FA05F4C5F120051EBFCB
:104CC00022FA05FC44EA0C04203556EA044C4FEA6B
:104CD000144418BF641C4FF000084FF000099042C4
:104CE00071EB030C39D3002919BFB1FA81F701FA2E
:104CF00007F6B0FA80F700FA07F6C7F120071EBFE3
:104D000020FA07FC46EA0C062037B6FBF4FCA7EBBA
:104D10000507103F07F01F0BCBF120060CFA0BFB29
:104D20002CFA06F644BFB3460026202FA4BF5E46E9
:104D30004FF0000B5BEA060C08BF4FF0010B19EBBC
:104D40000B09ABFB027C48EB0608C01B06FB02CC40
:104D50000BFB03CC71EB0C01C1E70B46024641464D
:104D60004846BDE8F08B13B54FF000004FF000014E
:104D7000AFF30080BDE81C407047B2F120030AD5B4
:104D8000C2F1200301FA02F120FA03F300FA02F063
:104D900041EA0301704700FA03F14FF00000704749
:104DA000B2F120030AD5C2F1200320FA02F001FA81
:104DB00003F321FA02F140EA0300704721FA03F0FD
:104DC0004FF00001704770477047704710B500F012
:104DD00009F8006810BD10B5044600F003F804603F
:104DE00010BD0000004870475C86002000487047F6
:104DF0005C8600207546FFF7F9FFAE460500694660
:104E0000534620F00700854618B020B5FBF7E4F9BB
:104E1000BDE820404FF000064FF000074FF00008BB
:104E20004FF0000B21F00701AC46ACE8C009ACE83C
:104E3000C009ACE8C009ACE8C0098D46704710B5A0
:104E40000446AFF300802046BDE81040FBF7AFB941
:104E500001491820ABBEFEE726000200704749005A
:104E600050EAC12018BF04204A0D18BF40F00100CD
:104E700040F2FF72B2EB515F08BF40F00200012820
:104E800008BF0520704700002DE9FF4D21F00048C4
:104E900007460C46B8F1795F08DA00F08BFF00286E
:104EA00001BF0020324904B0BDE8F08D3A462346E8
:104EB000104619460EF0C4F9054602462D480E4626
:104EC0000B460621784400F061FA2A4633460EF07C
:104ED000B7F9DDE9022382468B46384621460EF0BB
:104EE000AFF904460F4652465B46284631460EF05F
:104EF000A7F922463B460EF033FB07468A464FF0A1
:104F0000FF32284631460EF078FF1B4A90450ADAF8
:104F10003A4653460EF024FB04B00022BDE8F04DA3
:104F2000134B01F01CB8154A4245A8BFA8F500155F
:104F30004FF00004B8BF124D22462B460EF010FB76
:104F40000646884622462B46002009490EF008FBFB
:104F500004460D463A465346304641460EF000FBA5
:104F600004B022462B46BDE8F04D00F0F8BF00002B
:104F70000000F03F30F400003333D33F0000E93F3E
:104F80000000D23F01220EF038BF00221346104627
:104F9000114600F0B7BD0000024A002011070EF0D4
:104FA0002CBF000001FDFFFF2DE9F04106460F4632
:104FB0000EF0F0F9041E0D4618BF0120284320F022
:104FC0000040C0F17F6000F1E040C00F0ED0301C07
:104FD00018BF0120384320F00040C0F17F6000F18D
:104FE000E040C00F04BF0120FFF7F5FE2046294630
:104FF000BDE8F0810808A0F500114FEA31017047C3
:10500000080000002DE9F74F144694B00021C4E9D0
:1050100002111599079121F00045C9498D4206DC1E
:105020001599C4E9000117B00020BDE8F08FC5490B
:10503000DFF814A3A9423CDD0799C44E0029C44FF0
:10504000C44A1599534619DD0EF08AFA554506D023
:10505000C14AC24B0EF084FAC4E900010AE04FF0E5
:10506000D352BE4B0EF07CFA32463B460EF078FA35
:10507000C4E9000117B00120BDE8F08F00F092FCF8
:10508000554506D0B44AB54B00F08CFCC4E900018C
:105090000AE04FF0D352B14B00F084FC32463B465D
:1050A00000F080FCC4E9000117B04FF0FF30BDE80C
:1050B000F08FAB49A942159978DB21F00041834676
:1050C0008846A84AA84B0EF0BBF80022A74B00F078
:1050D00069FC00F06FFE099000F0C9FE06460F461D
:1050E0009C4A53460EF0ACF843465A4600F037FF50
:1050F00080468A46984A994B304639460EF0A0F8C9
:105100002A0D01250B924246534600F028FF032D3D
:10511000C4E9000139D00B98C1F30A51401A05EBDC
:1051200045111139814230DA9148C346784400EB89
:105130000510CDF80CA00C90D0E90023304639467C
:105140000EF07EF802460B460491069058460399ED
:105150000EF006FA80468A4602460B4658460399E8
:105160000EF0FEF9049B069A0EF0FAF983460C98AD
:1051700003913946D0E9022330460EF061F85A46D1
:10518000039B0EF0EDF96D1CBDE707980028A2BF48
:10519000099817B0BDE8F08F616881F00041616047
:1051A000099817B04042BDE8F08FFFE78446159894
:1051B000C1F31301C0F30A50A0F2F5304FEA6018B2
:1051C00000F01F06C6F12000139000200690079003
:1051D00041F4801E05206D4676B1664A08EB000159
:1051E0007A4452F8213002EB8101B3404A681399A6
:1051F00022FA01F1194305E05F4908EB0002794406
:1052000051F82210A1FB0E27A1FB0C131A449A425D
:1052100034BF0123002303EB070A05EB8003D3E926
:1052200001B70F448F4234BF0121002193448B44C6
:1052300011B1934502D903E0934501D2012100E069
:105240000021C3E901B7514445F82010011EA0F127
:105250000100C1DC0298059F00F10050800F129000
:105260000298DDE90356800000F001FE83462846DF
:105270000D9100F013FE6FF01D020EF0BEFDCDE9A2
:105280000E01304600F00AFE6FF03D020EF0B5FD53
:1052900080468A46384600F001FE6FF05D020EF04F
:1052A000ACFD074642465346119100F07BFBDDE919
:1052B0000E2300F077FB5A460D9B00F073FB002590
:1052C0000E465A4628460D9B0EF04AF9DDE90E239C
:1052D0000EF046F9424653460EF042F93A46119B0B
:1052E00000F03DFEDFF898A0244A53460DF0A8FFD9
:1052F00007468846234A244B314628460DF0A0FF36
:105300003A46434600F04EFB074688464FF0A84217
:105310005346314628460DF093FF3A46434600F087
:1053200041FB159A12F0004F04D0129A81F000410F
:1053300052421292C4E90001129817B0BDE8F08FF2
:10534000FB21E93F7CD90240FB21F93F7370032E1A
:105350008A19A33B000040543163621A61B4D03D06
:10536000FB21394183C8C96D305FE43F0000E03F55
:10537000F8F1000074F1000056F10000182D4454BB
:10538000FB21F93D3326A611460B113C2DE9F041D6
:105390004F1E00EBC7010446D1E9000115461E4629
:1053A00037F006020DD02A4633460DF049FF7F1E26
:1053B00004EBC703D3E9002300F0F4FA37F0060248
:1053C000F1D1022F25D0042F13D0062F18BFBDE82E
:1053D000F0812A4633460DF033FFD4E90A2300F06A
:1053E000E1FA2A4633460DF02BFFD4E9082300F0FA
:1053F000D9FA2A4633460DF023FFD4E9062300F0FC
:10540000D1FA2A4633460DF01BFFD4E9042300F0FD
:10541000C9FA2A4633460DF013FFD4E9022300F0FF
:10542000C1FA2A4633460DF00BFFD4E90023BDE84C
:10543000F04100F0B7BA00002DE9FF4D054621F01C
:10544000004084B00C46B0F1795F0BDA2846FFF7D4
:1054500006FD042808BFFFF79FFD284608B0214637
:10546000BDE8F08D2A460B4610460DF0E9FE0646D3
:105470000F462A4623460DF0E3FE804626488A461C
:1054800032463B4605217844FFF780FF834610985B
:10549000029160B3214A224B404651460DF0D0FEA6
:1054A000CDE900015A4640465146029B0DF0C8FE28
:1054B00082468846DDE906014FF0FF320EF09DFC82
:1054C000524643460EF04CF832463B460DF0B8FECD
:1054D000DDE906230EF044F8DDE900230EF040F884
:1054E00008B02A462346BDE8F04D00F038BD0B4613
:1054F0005A46304639460DF0A3FE084A084B00F0E4
:1055000051FA424653460DF09BFE08B02A46234608
:10551000BDE8F04D00F046BA66EF0000495555551C
:105520005555C5BF2DE9F04D04468CB0904821F08B
:105530000047164698460D460991874206DA2046EE
:10554000294600F037FC002800F0AE808948B842B8
:105550001CDC09980028BCBF85F0004588F0004895
:10556000854A864B2046294600F0F9FC04460D4644
:1055700032464346824883490DF0F2FF22462B46CD
:1055800000F010FA002604460D46B04622462B468F
:10559000104619460DF054FE8B46824602460B46D5
:1055A0000DF04EFE0246089077480B46009106210A
:1055B0007844FFF7EBFECDE90310744806217844E8
:1055C000009B089AFFF7E2FE52465B460DF038FE5C
:1055D000CDE9051052465B46204629460DF030FEC7
:1055E00007910090DDE90310DDE9053200F0DAF9FA
:1055F000079B009A0DF024FE3246434600F0D2F994
:1056000052465B460DF01CFE3246434600F0CAF996
:1056100080460E465E4A5F4B079900980DF010FEDB
:105620004246334600F0BEF982468B4622462B4660
:1056300000F0B8F980464F480E46B84214985BDC3B
:1056400000F015FC074642463346059100F0AAF9E2
:10565000CDE9011042463346104619460DF0F0FDE3
:10566000DDE9013200F04EFA52465B460DF078FF5C
:1056700022462B4600F073FC01220EF0BEFB3A4698
:10568000059B00F06CFC04460D460998022101EAD6
:10569000A070C0F1010000F0EAFB0CB022462B46DE
:1056A000BDE8F04D0DF0CCBD1498401C38432043AC
:1056B0000BD01498012812D00CB022462B46BDE81E
:1056C000F04D0020344900F01DBA0CB025F0004325
:1056D0002246BDE8F04D0020304900F013BA2046C4
:1056E0002946FFF7BCFB042808BFFFF755FC2046FE
:1056F0000CB02946BDE8F08D012802BF40460CB031
:10570000BDE8F08D00270B463A462046294600F0BA
:1057100026FC52465B4600F022FC04460D464246FB
:10572000334600201C4900F0EDF983463A4688468E
:10573000334610460DF084FD0022184B00F032F97C
:1057400006468A4622462B46384641460DF078FDED
:105750003246534600F026F95A4643460DF070FD96
:105760000CB03A464346BDE8F04D00F01BB90000CE
:105770000000303E2894E53F182D4454FB21E93FBA
:10578000075C143326A6813C64EE000086EE000020
:10579000635555555555D53F0000F0BF0000F03F0B
:1057A00000B5244B21F0004287B09A42DCBF0022B2
:1057B000134629DD204B9A4208D140B94FF0010031
:1057C000FFF709FBFFF7E1FB07B000BD03DBFFF7C5
:1057D000D9FB07B000BD02AAFFF714FC10F00301CB
:1057E00004BF0DF1080C9CE80F000DD00120012929
:1057F0000ED0022914D00DF1080C00909CE80F0087
:10580000FFF71AFE07B000BDFFF73EFB07B000BD73
:105810000DF1080C00909CE80F00FFF70DFE05E06D
:105820000DF1080C9CE80F00FFF72EFB07B081F08C
:10583000004100BDFB21E93F0000F07F00B5254B92
:1058400021F0004287B09A4203DC00221346009206
:105850002BE0214B9A4208D140B94FF00100FFF7ED
:10586000BAFAFFF792FB07B000BD03DBFFF78AFB34
:1058700007B000BD02AAFFF7C5FB10F003014FF00F
:1058800001000DD0012914D002291AD00DF1080C05
:105890009CE80F00FFF7F8FA07B081F0004100BD67
:1058A0000DF1080C00909CE80F00FFF7C5FD07B054
:1058B00000BD0DF1080C9CE80F00FFF7E5FA07B0FA
:1058C00000BD0DF1080C00909CE80F00FFF7B4FD3F
:1058D000E2E70000FB21E93F0000F07F10B5164B26
:1058E00021F00042012486B09A4203DC00221346D4
:1058F00000941CE0114B9A4208D140B94FF00100CE
:10590000FFF769FAFFF741FB06B010BD03DBFFF7B5
:1059100039FB06B010BD02AAFFF774FB00F00100CE
:10592000A4EB40000DF1080C00909CE80F00FFF77D
:10593000F9FD06B010BD0000FB21E93F0000F07F3B
:1059400021F00042A2F16052B2F5801F01F0004345
:1059500028BFD2F17F6C0BD95FEA001C43EAC20278
:1059600042EB507018BF704728BF20F0010070470D
:10597000B2F5801FBCBF184670474FEA410C1CF5BA
:10598000001F02D2084600F02CBB70B500F099FA57
:1059900000000089FFF7F6BF4FF00040A0F580003F
:1059A0007047000010B591EA030F48BF83F0004331
:1059B0000DF1DE85841A71EB030C05D2121943EB4D
:1059C0000C03001B61EB0C01DFF824E14FEA1154DA
:1059D000A4EB135C1EEA430F18BF9EEA445F73D02A
:1059E00023EA0E03DCF1200E21EA045143F4801374
:1059F00032D322FA0CFE10EB0E0023FA0CFE41EB20
:105A00000E01CCF1200E03FA0EFE10EB0E0051F148
:105A10000001B1F5801FCCF1200E32D201EB045110
:105A200012FA0EF2BDE8104058BF7047401C38BF54
:105A30005FEA420218BF7047002814BF20F001003F
:105A400041F100014FEA410313F5001F38BF7047D1
:105A5000A1F1C041FFF7CEBA012A43EB0302ACF13A
:105A6000200CDCF11F0E32BF4FF0000E23FA0CF3B6
:105A700010EB030041EB0451B4EB115FD0D0A1EB6C
:105A8000045101F5801149085FEA300001EB04512F
:105A90000ED350F1000038BF12FA0EFE08D1BDE857
:105AA0001040C9E7401C38BF5FEA4202CAD1C3E7D1
:105AB000BDE810404FEA410313F5001F38BF70479F
:105AC000A1F1C041FFF796BA9EEA445F08D011EAFF
:105AD0005E0FBDE8104004BF01F000410020704798
:105AE000BDE8104070B500F0ECF900BF64FBBE3EAD
:105AF0000000E0FF02494FF000000EF04CB900BF7B
:105B00000000F87F2DE9C04130B4DFF8A0C23CEAC4
:105B1000111418BF3CEA131400F0EC8081EA03056D
:105B20001CEA111444EAD57418BF1CEA131500F0DE
:105B3000C780A4EB05044FF0004545EAC12145EAC2
:105B4000C32341EA505143EA525304F17F7499420E
:105B500004F500344FEAC0204FEAC22208BF904249
:105B600000F09C804FEA13650FF24016765D4FEA15
:105B7000134506FB05F7C7F1807706FB07F74FEAE9
:105B8000D737A7FB03687642C8F58038A7FB06CE57
:105B900038BFA8F1010807FB08E64FF0000EA6FB8E
:105BA000028CE6FB03CEDCF1000CCEF1004E38BFD8
:105BB000AEF1010EA6FB0C584FF000074FF00005A8
:105BC000E6FB0E87A1FB08C6A0FB07CE16EB0E0670
:105BD00045F10005E1FB076515F1E04E7EBFA4F538
:105BE00080345FEA46066D4116F1800745F10005F5
:105BF0004FEA17274FEA066647EA0567A6F1DE4631
:105C0000B6F1805F4FEA15251FD9384624F0010C04
:105C100005EBC471BCF1FE6F01EB0C1102D8F0BCB6
:105C2000BDE8008124425CBF01F5801E9EEAC47F6E
:105C300002D4F0BCBDE80081244238D4F0BCA1F10C
:105C4000C041BDE80041FFF7D5B94FEAD22242EA90
:105C500043524FEAD323A7FB02864FEAD02040EA03
:105C6000415007FB03661EEA0E0F4FEAD12105FBE8
:105C7000026658BFA6EB0056B6EB00564FEA520E2E
:105C80004EEAC37E18EB0E0E56EB530EBDD518EB45
:105C900002085E417F1C55F10005B6E74FF4801500
:105CA0004FF000074FF000064FF00008ADE7F0BCE2
:105CB0004FF0000001F1C04101F00041BDE800815A
:105CC00011EA0C1F0CEA131500D00CE013EA0C1FAC
:105CD00000F025804FF00000F0BC81EA030101F0E4
:105CE0000041BDE80081F0BCBDE8004181EA03014C
:105CF000FFF780B9F0BCBDE8004170B500F0E1F8F5
:105D0000097EFC3E00F007B881EA03014FF0000075
:105D100001F00041704781EA0301FFF76BB9F0BC65
:105D2000BDE800414FF0000021497047FFFDFBF93D
:105D3000F7F5F4F2F0EEEDEBE9E8E6E4E3E1E0DEBE
:105D4000DDDBDAD8D7D5D4D3D1D0CFCDCCCBCAC830
:105D5000C7C6C5C4C2C1C0BFBEBDBCBBBAB9B8B757
:105D6000B6B5B4B3B2B1B0AFAEADACABAAA9A8A84A
:105D7000A7A6A5A4A3A3A2A1A09F9F9E9D9C9C9B18
:105D80009A999998979796959594939392919190C3
:105D90008F8F8E8E8D8C8C8B8B8A89898888878754
:105DA0008685858484838382828181800000FF07C9
:105DB0000000F87F4FEA41034FEA5353A3F5806395
:105DC000D3F11E03C8BFD3F1210C0CDD4FF000420C
:105DD00042EAC12242EA505232FA03FC8CEAE17CE8
:105DE000ACEBE1707047102BC4BF0020704703F587
:105DF000787CBCF1FF3F04D06FF0004282EA2100C2
:105E0000704770B500F05DF849922480002070471B
:105E1000F2E700004FEA1153A3F58063D3F11E03AC
:105E2000A8BFD3F1200C08DB4FF0004242EAC122A8
:105E300052EA505232FA03F0704709420BD4102B49
:105E4000C4BF0020704703F5787CBCF1FF3F05D04C
:105E50004FF0FF3070474FF00000704770B500F012
:105E600030F800BF4992248000207047F0E710F01E
:105E7000004248BF4042B0FA80F310FA03F10AD062
:105E8000C3F11D0303F580634FEA415002EB035257
:105E900002EBD12170474FF000007047B0FA80F359
:105EA00010FA03F10AD0C3F11D0303F580634FEA32
:105EB00041504FEA035202EBD12170474FF00000EE
:105EC00070470EF1020E2EF0030E5EF8046B3642A0
:105ED00005D4012A43EB030515F5001F12D801284C
:105EE00041EB010C1CF5001F0CD80ED14FEAD17C00
:105EF00015F5001F0CEB4C0C0CF1020C08BF4CEB21
:105F0000D37C04E04FF0080C01E04FEAD37C0CEBAB
:105F10004C0526FA05F606F00706B6F1040C06D283
:105F20000EEB860CBDE870404CF0010C6047DFE8DA
:105F30000CF0090B02024FF000414FF00000A1F5F8
:105F4000002170BD19461046012851EB010418BF0D
:105F5000D4F5001484BF002001F0004170BD91EA27
:105F6000030F10B581F000413FF524AD83F00043ED
:105F70000DF0FEBA43004FEAD30C4FEA3C0C43400D
:105F80001FBF40070CF1605113F0FE4F70471CF02B
:105F9000006F03D100200CF0004170470CF000436B
:105FA00043EA507010B540EACC000DF008FE00BF87
:105FB000000000924FEA0001FFF71CB84FF00041CB
:105FC0004FF00000A1F500217047401058BFC0F10C
:105FD0004040491058BFC1F140418142EFF3008079
:105FE0007047FF2141EAD050C00570470102040804
:105FF00010204080FEFDFBF7EFDFBF7F00000000B8
:106000001000D8BA000000002020202020202020EE
:106010002020202020202020202020202020202080
:106020002020202020202020202020202020202070
:10603000F409FF0BF401E703640EC70EDC0EFF0E3C
:106040009001FE03000000000000000000000000BE
:106050008300000000000000000000000F00FFFFB0
:10606000FFFFFFFFFFFFFFFFFFFFFFFFFFFFFFFF40
:10607000FFFFFFFFFF000000000000000000000025
:106080000000000000000000000000000000000010
:106090000000000000000000000000000000000000
:1060A00000000000000000000000000000000000F0
:1060B00000000000000000000000000000000000E0
:10E4D00030B50024012512E00B185B1E5B089A4240
:10E4E00006D81DB9091A491C04EB51041946F1E775
:10E4F0001DB1081A401C04EB5004581C002588422A
:10E50000EAD3204630BD70B50025012310E00C1A77
:10E51000641C05EB5404A24201D2012600E000264F
:10E520009E4208D003B125460844401C4008002301
:10E530008842ECD370BD03B925460144491E490801
:10E54000E3E70346012101E05B084900002BFBD112
:10E5500019B102460020491EBAE74FF0FF3070475C
:10E560000346012101E05B084900002BFBD119B1F2
:10E5700002460020491EC6E74FF0FF30704770B5D5
:10E58000FD4CFE4DA06D2844C0F34F0004F05AF836
:10E5900000286079FA494FEAC07001D0A8B126E09E
:10E5A000002811D0A06D42195010C31700EB537012
:10E5B00001EBE00120F00700C0EB6200F14A0B78AC
:10E5C000805C03430B70012070BDA06D4219501098
:10E5D000C31700EB537001EBE00120F00700C0EB24
:10E5E0006200E84A0B780832805C03400B70002020
:10E5F00070BDE5480022A0F8182EB0F8882E4AB960
:10E60000A0F8861EDC49DD4AC96D521E1144490836
:10E61000A0F8881EB0F8881EA0F88A1E704770B552
:10E62000DA4BD54903EBD00200F007050846D54C7C
:10E63000407912784006655D0E7B000E2A40012E5F
:10E64000487101D05AB970BD002AFCD00A8C03EB86
:10E65000D20302F007021B78A25C1342F3D040F011
:10E660000100487170BD70B5C84BC34903EBD002BF
:10E6700000F007050846C34C407912784006655DF6
:10E680000E7B000E2A40012E487102D0002A0ED1C6
:10E690000AE0002A0BD10A8C03EBD20302F0070236
:10E6A0001B78A25C134202D040F00100487170BD9B
:10E6B000B64A02EBD00100F007000A78B149085CC5
:10E6C0000242AD48417904D0CA0702D041F00101AD
:10E6D00001E001F0FE0141717047AC4A02EBD0014C
:10E6E00000F007000A78A749085C0242A248417975
:10E6F00004D1CA0702D041F0010101E001F0FE019E
:10E7000041717047A14A02EBD00100F007000A787E
:10E710009C49085C02409848417952EAC17202D093
:10E7200041F0010101E001F0FE0141717047974A9B
:10E7300002EBD00100F007000A789249085C024021
:10E740008D48417901F001035B1E1A4202D141F06C
:10E75000010101E001F0FE0141717047F0B5864B07
:10E76000884E19465F7B4D7988490836854C00F004
:10E77000070201EBD001012F30D11F7B012F04D004
:10E780000A282BD2E8072BD1F0BD7B4FDFF8FCE144
:10E790000A28B7F820C00CF007070EEBDC0C08D2F3
:10E7A000E807F1D09CF80000F35D18408CF80000F9
:10E7B00016E09CF800C0E75D1CEA070FE4D0ED0707
:10E7C00012D00D78A25C15430D70714A997B22F826
:10E7D0001100491C9973F0BD0870F0BDE80703D023
:10E7E0000878A25C1043F7E70878B25C1040F3E7C2
:10E7F0002DE9F04760494A79D2070ED00D7B634A74
:10E80000DFF8809100F0070402EBD003012D06D061
:10E81000187819F8041008431870BDE8F087594DAE
:10E8200000208E7B0835DFF868A10FE03AF810C0B1
:10E83000401C02EBDC070CF0070C97F8008015F881
:10E840000CC0C0B208EA0C0887F80080B042EDD9CD
:10E85000088C02EBD00200F007001678285C064016
:10E860001670187819F80420104318700020887367
:10E87000D3E710B540490122444C4A730A73088417
:10E880004A7904EBD0035206120E3E4C4A7100F056
:10E8900007001B78205C034202D042F0010048715F
:10E8A00010BD70B43449F83808284A798D7902F0DF
:10E8B000FE0405F0010644EA060320D2DFE800F07A
:10E8C00004091014161A1F0E42F0FE0000EA52004E
:10E8D00003E002F0010040EA5200487170BC70474A
:10E8E00065F35F028A71F9E74B71F7E74B716808CE
:10E8F0008871F3E70120904304434C71EEE770BC4C
:10E9000002214FF4746074E62DE9F0411A4C1D4F5A
:10E910001A4E60791A4DC107204607F10807806D2D
:10E9200030443DD0C0F34F0003F08CFE174A6FF423
:10E93000D05158B1A06D008801EAD001114400F017
:10E9400007000A78385C02400A7037E0A36D1E4465
:10E950007010C71700EB577005EBE00520F00700BB
:10E96000C0EB660607482F78365C37432F701B884C
:10E9700001EAD30111440DE030000020A49FFFF70D
:10E98000CD070020EC5F00080010002000100020E0
:10E99000AC05002003F007030A78C05C0243D3E70C
:10E9A0004110CA1701EB527105EBE10221F007019A
:10E9B000C1EB60001378C05D03401370A06D801C34
:10E9C000A065BDE8F0812DE9F041F84CFA4DF84E14
:10E9D0006079F84FC1072046806D2844C0F34F008E
:10E9E00013D003F02FFEC0BBA06D41194810C21711
:10E9F00000EB527006EBE00220F00700C0EB610074
:10EA00001378C05D0343137032E003F01BFEE94B43
:10EA1000EA4A08330028A06D6FF4D0511ED0054497
:10EA20004FEA650C4FEAEC7E0CEB5E7C06EBEC06E5
:10EA30002CF0070CCCEB650596F800E0EB5C0EEAD9
:10EA4000030E86F800E0008801EAD001114400F0CE
:10EA500007000A78385C024309E009E0008801EA0F
:10EA6000D001114400F007000A78185C02400A70D7
:10EA7000A06D801CA065A4E72DE9F041DFF82CC350
:10EA80000B46A0F1820EDCF8601041EA0221BCF8CE
:10EA9000102011444FF6FC7201F01F0502EAD10666
:10EAA000CCF860100021BEF10F0F59D2DFE80EF054
:10EAB000085811581C5826582F58385842584C009E
:10EAC00003F00F002A46F6F758F903460F460F20C9
:10EAD00006E0D8B22A46F6F750F903460F46FF2063
:10EAE000A840C043C41740E0C3F30B002A46F6F722
:10EAF00044F903460F4640F6FF70F1E798B22A4604
:10EB0000F6F73BF903460F464FF6FF70E8E7C3F30D
:10EB100013002A46F6F731F903460F46A848DFE707
:10EB200023F07F402A46F6F728F903460F466FF098
:10EB30007F40D5E723F070402A46F6F71EF90346DA
:10EB40000F466FF07040CBE718460C462A46F6F7A2
:10EB500014F903464FF0FF30A8400F46C04304E0CD
:10EB6000DCF85810891DCCF858109449725831447B
:10EB70000240924849681A43325021403044394398
:10EB800041601EE7894910B50A6E4FF6FC7342EAF0
:10EB900000200A8A104400F01F02086603EAD0032E
:10EBA0004A828B8285498548194418584968F6F786
:10EBB000F7F810BD30B57D498A6D32F8023B1C0A6A
:10EBC000803C092C15D2DFE804F005140B14161450
:10EBD0001C14220000EB032080B24FF4E06304E039
:10EBE00000EB032080B24FF4006303EB5000C882B7
:10EBF0008A65C88A30BD00EB032080B24FF4A06361
:10EC0000F3E700EB032080B24FF48053EDE700EB15
:10EC1000032080B241F2E833E7E710B5634CA16D01
:10EC200031F8020B020A842A02D0862A11D10AE0A6
:10EC3000C0B2607011F8022B40EA0220208300204D
:10EC4000A165207005E0C0B26070A165FFF7B2FF5A
:10EC50002083208B10BD70B5544C4FF6FF75A06D0E
:10EC600030F8023BA065028803F47F41DBB205EA7D
:10EC70000225236641EA12212B43A1F50645803D7A
:10EC800031D0A1F50645823D2FD0A1F50645843D42
:10EC90002FD0A1F50645863D2FD0A1F50645883D2C
:10ECA0002DD00025A1F5044082382AD0A1F50440DA
:10ECB00084382CD0A1F5044086382DD0A1F504402D
:10ECC00088382FD0A1F504408A3830D0A1F504400F
:10ECD0008C3832D0A1F504408E3834D0A1F50440F0
:10ECE000903836D03DE0374904E003F12023A36299
:10ECF00035E035491944A16231E03449FAE7344935
:10ED0000F8E7D0B2FFF73EFF00F00F0024E0D0B2EA
:10ED1000FFF738FFC0B21FE0D0B2FFF733FFC0F3F8
:10ED20000B0019E0D0B2FFF72DFF80B214E0D0B293
:10ED3000FFF728FFC0F313000EE0D0B2FFF722FF69
:10ED400020F07F4008E0D0B2FFF71CFF20F07040B9
:10ED500002E0D0B2FFF716FFA0622570A06D801C04
:10ED6000A065A06A70BD1B49800B07D0012808D0A0
:10ED7000022809D003280AD000207047B1F83A0EC3
:10ED80007047B1F86E0F7047B1F8720F7047B1F865
:10ED9000760F70470F49800B1ED001281FD0022824
:10EDA00020D0032821D00020704700003000002030
:10EDB000CD070020EC5F0008A49FFFF700100020A3
:10EDC000FFFF0F00001E0020001A0020003000206E
:10EDD000D037002000100020B1F87A0FE4E7B1F836
:10EDE0007E0FE1E7B1F8820FDEE7B1F8860FDBE7CF
:10EDF000F849800B07D0012808D0022809D0032841
:10EE00000AD00020D0E7B1F8380ECDE7B1F86C0F8A
:10EE1000CAE7B1F8700FC7E7B1F8740FC4E7ED495E
:10EE2000800B07D0012808D0022809D003280AD077
:10EE30000020B9E7B1F8780FB6E7B1F87C0FB3E777
:10EE4000B1F8800FB0E7B1F8840FADE7810BE1486E
:10EE500007D001290AD002290DD0032910D00020A3
:10EE6000A2E7B0F8381EB0F83A0E0DE0B0F86C1F0B
:10EE7000B0F86E0F08E0B0F8700F00EB004093E7B9
:10EE8000B0F8741FB0F8720F01EB00408CE7810BF3
:10EE9000D0480AD001290DD002460229B2F8822FAB
:10EEA0000FD0032910D000207EE7B0F8781F90F82B
:10EEB0007A0F03E0B0F87C1F90F87E0F01EB004062
:10EEC00006E0B0F8800F01E0B0F8840F00EB0240DC
:10EED00080B269E72DE9F047BF4CDFF80093DFF817
:10EEE0000083A26D32F8021BA265108801F47F43F3
:10EEF00043EA10254FF6FF7303EA0026CBB22366E0
:10EF000033434AF28746A91BB5426FD043DCB24F68
:10EF100048F2826CA5EB0C06796E3F8A65456CD091
:10EF200021DC48F28A48A5EB080C4FF00106454564
:10EF300059D00BDCA5F28245B5F5004541D0022D34
:10EF400042D0042D49D0062D79D149E0BCF1020F01
:10EF500049D0BCF1040F46D0BCF1060F43D0BCF53C
:10EF6000FB7F6CD143E041F6016CA6EB0C006645DB
:10EF70006DD009DC022E47D0042E4BD0062E4ED089
:10EF8000B6F5F05F5BD15EE001285CD002285ED070
:10EF9000032854D157E00A2959D008DC0A294ED257
:10EFA000DFE801F04D515551555155515551A1F2E0
:10EFB000FB11082943D2DFE801F04E5260647377F9
:10EFC0008488C2B2822001E0C2B28420FFF754FDDF
:10EFD000A06D801CA065667231E0C2B28620F5E7A4
:10EFE000C2B28820F2E7C2B2E8B2EFE72FE03B44BA
:10EFF00003EB0900C0F8001E03E0D81900F120203F
:10F000000BE0921CA2651AE03B4403EB0900C0F838
:10F01000001AF6E73B4403EB08000160F1E73B44CC
:10F0200003EB0800C0F8D017EBE72066E8B2C3F3A3
:10F030000522616EFFF720FDA06D801CA065A06D0C
:10F04000001DA06514E41846FFF700FFEDE7184621
:10F05000FFF71DFFE9E71846FFF7F8FE02E0184644
:10F06000FFF715FFC3F30D0101EB4000B4F8641086
:10F0700000F1202089B20160DEE71846FFF7E6FEC6
:10F0800002E01846FFF703FFC3F30D0101EB400157
:10F09000B4F8640082B201EB0900C0F8002ACBE7A3
:10F0A0001846FFF7D3FE02E01846FFF7F0FEC3F361
:10F0B0000D0101EB4001B4F8640082B241F8082070
:10F0C000BAE71846FFF7C2FE02E01846FFF7DFFE78
:10F0D000C3F30D0101EB4001B4F8640082B201EB0F
:10F0E0000800C0F8D027A7E72DE9F05F3A4CDFF819
:10F0F000ECA0DFF8EC90A06D4FF4FD7B30F8021B24
:10F10000A065B0F8008001F47F4242EA18234FF670
:10F11000FF7202EA0825CAB222662A4349F28565CF
:10F12000591BAB427DD05DDC49F28345A3EB050161
:10F13000AB423FD033DC284D48F2826CA3EB0C0786
:10F14000696E2D8A0EB263456CD01EDC48F2864C87
:10F15000A3EB0C074FF0010963456ED00BDCA3F263
:10F160008243B3F5004369D0022B68D108F0FF0257
:10F1700089B284209EE0022F5FD05F455FD12A4490
:10F1800002EB0A01A1F8006E04E1022F76D0042FF1
:10F1900075D0062F74D0B7F5606F50D1B4E0052953
:10F1A0006FD008DC01296CD0022903D0032968D074
:10F1B000042944D1ADE0062970D0A1F58071FF3952
:10F1C0006DD001296CD002297BD11046FFF7CBFD11
:10F1D000BCE00000001000203000002000100020E3
:10F1E0000030002040F60365A1F60360A94223D059
:10F1F0002FDC40F6FE55A1F6FE50A94228D01FDCB8
:10F2000003296FD012DC01296DD0022959D1104693
:10F21000FFF7C0FDC2F30D0101EB4002B4F864003A
:10F2200001E090E04FE022F80900B2E004296FD03D
:10F23000A1F55061FD3944D1AFE037E031E040E065
:10F2400001286ED0022803D003286AD0042838D1C0
:10F25000A7E040F2FD15A0F2FD11A8426FD011DC2D
:10F2600001286DD058456CD0A0F58070FB3869D06E
:10F27000012826D11046FFF7BBFD67E027E02CE010
:10F2800032E041E0012970D002296FD003296ED00D
:10F29000042916D11046FFF7C2FD70E039E03CE0CA
:10F2A00040E008F0FF0289B2822003E008F0FF028C
:10F2B00089B2D8B2FFF7E0FBA06D801CA06584F88E
:10F2C0000990BDE8F09F511901F1202108E02A447E
:10F2D00002EB0A01A1F8006A5CE02A4402EB090192
:10F2E0000E8057E044E03CE02A4402EB0901A1F81B
:10F2F000D0674FE02066B4F86400C2F3052281B203
:10F30000D8B2FFF7B9FB44E01046FFF72CFDF1E758
:10F3100032E01046FFF73EFDECE71046FFF723FD15
:10F3200003E03AE01046FFF735FDC2F30D0101EBB3
:10F33000400000F12020B4F86410018029E03CE096
:10F340002FE032E035E01046FFF724FDC2F30D0157
:10F3500001EB400202EB0A01B4F86400A1F8000AD4
:10F3600017E01046FFF7FFFC54E72AE02DE030E0FD
:10F370001046FFF7F8FC02E01046FFF70BFDC2F362
:10F380000D0101EB400202EB0901B4F86400A1F8A1
:10F39000D007A06D801CA06593E71046FFF728FDFD
:10F3A000A8E71046FFF73BFDA4E71046FFF720FD56
:10F3B000BBE71046FFF733FDB7E71046FFF72FFD19
:10F3C000C4E71046FFF714FD24E71046FFF727FDBA
:10F3D00020E71046FFF70CFDD1E72DE9FE4FF84C72
:10F3E00049F28467DFF8DC93A16D31F8022BA16547
:10F3F00002F47F430888D2B243EA10264FF6FF7327
:10F4000003EA002322661A43F51BEF4BBE427CD071
:10F410007CDCEE4D49F28708A6EB080CB5F83A7E85
:10F420000297B5F86E7F0197B5F8727F0097B5F82F
:10F4300076EFB5F87ABFB5F87EAFB5F8827FB5F84C
:10F44000865F464571D049DCDD4D48F28668A6EB03
:10F45000080C2D8A464569D023DC48F2864CA6EB81
:10F460000C074FF00108664577D00EDC06F5FF4625
:10F47000B6F5803672D0B6F5007F6FD0A6F58066FF
:10F48000023E6CD0022E6BD108E1022F69D0B7F595
:10F49000FD7F67D0B7F5FE7F48D0B7F5FF7F5FD11E
:10F4A00027E140F6FD16ACF6FD10B44532D00EDC77
:10F4B000BCF1020F7ED0ACF5006CBCF5FD7C7AD0BF
:10F4C000BCF1010F78D0BCF1020F49D1B0E10128A5
:10F4D00073D0022872D0032842D123E1BCF57F7F8C
:10F4E0006DD024DC40F2FD13ACF2FD109C4564D0DD
:10F4F00011DCACF5807CBCF1F90C5CD0BCF1010FE7
:10F500005AD0BCF1020FE1D001E063E135E0BCF17B
:10F51000030F25D1FDE0012850D002287DD003281B
:10F5200003D0B0F5FF7F1BD106E1FFE0DCE040F245
:10F530000141ACF201408C4570D014DCACF5407C4C
:10F54000BCF1FD0C6BD0BCF1010F69D0BCF1020F16
:10F5500067D0BCF1030F03D112E1AFE096E097E072
:10F560007FE0B1E0B4E0012879D0B0F5FD7F77D03D
:10F57000A0F58070FB3874D11EE1944E40F6014C2A
:10F58000A5F60140B6F87C7F0097B6F880EFB6F894
:10F5900084BF65456FD04CDC8C48B5F5206FB0F862
:10F5A00038AEB0F86CCFB0F8707FB0F8746FB0F8C8
:10F5B000780F05E0A3E0BBE0BCE099E02CE0BFE001
:10F5C00036D016DC052D74D008DC012D72D0022D4A
:10F5D00071D0032D70D0042D43D113E1A5F5106532
:10F5E000FC3D19D0012D68D0022D16D0032D77D106
:10F5F0001BE140F6FD38A5F6FD3345455DD011DC35
:10F60000A5F52065013D36D0012D70D0022D6FD0BB
:10F61000A5F58075FB3D63D181E075E0BBE09DE021
:10F62000A0E0A9E0012B7DD0022B6ED0032B57D197
:10F630006DE0B0F5017F69D01EDC40F2FF15A0F24D
:10F64000FF13A84270D00DDC012862D0022863D0DD
:10F65000A0F58070FD3868D0012841D1EEE09EE031
:10F66000A6E025E0012B76D0022B75D0032B74D0B9
:10F67000042B35D1FEE0DBE0A0F2FD3008282FD2CC
:10F68000DFE800F0EFEEEDECEBEAE9E8628325E07D
:10F69000C0B2FFF777FA00F00F0003E0C0B2FFF747
:10F6A00071FAC0B2608384F80A80A06D801CA065E6
:10F6B00016E0ABE092E09DE0A0E0B3E0C0B2FFF75F
:10F6C00061FAC0F30B00EDE7C0B2FFF75BFAE9E7C0
:10F6D0002A4402EB0900B0F8000EA7E0891CA165DE
:10F6E000B4F91A00BDE8FE8F5019C05A9EE010E030
:10F6F00012E02A4402EB0900B0F8000A96E0501923
:10F700001844B0F8D00791E00CE08EE0B6E0104469
:10F710008CE00EEB020089E00BEB020086E00AEBC6
:10F72000020083E0B81881E08CE083E0A8187DE057
:10F730000298ECE70198EAE71046FFF714FB02E0B5
:10F740001046FFF727FB2066C2F30520FFF71AFAE1
:10F7500000F00F0064E079E084E087E01046FFF7F6
:10F7600002FB02E01046FFF715FB2066C2F30520FE
:10F77000FFF708FAC0B253E01046FFF7F4FA02E0D0
:10F780001046FFF707FB2066C2F30520FFF7FAF9E2
:10F79000C0F30B0044E01046FFF7E5FA02E0104624
:10F7A000FFF7F8FA2066C2F30520FFF7EBF937E020
:10F7B0001046FFF7D8FA6CE01046FFF7EBFA68E066
:10F7C0003000002000100020003000200010002039
:10F7D000008825E01046FFF7C6FA02E01046FFF762
:10F7E000D9FAC2F30D0101EB400101EB0900B0F8B9
:10F7F000000A15E01046FFF7B6FA60E01046FFF782
:10F80000C9FA5CE01046FFF7AEFA02E01046FFF7D7
:10F81000C1FAC2F30D0101EB40001844B0F8D00763
:10F82000608342E70CEB020000E0B018608355E70C
:10F8300000986CE71046FFF7DBFA84E71046FFF705
:10F84000EEFA80E71046FFF7D3FA8EE71046FFF78F
:10F85000E6FA8AE73DE038E02EE029E024E01FE008
:10F8600014E00FE01046FFF7C3FA8CE71046FFF7ED
:10F87000D6FA88E71046FFF7BBFA93E71046FFF782
:10F88000CEFA8FE71046FFF7B3FA02E01046FFF713
:10F89000C6FAC2F30D0101EB400000F1202097E70A
:10F8A0001046FFF7A5FA9CE71046FFF7B8FA98E76D
:10F8B0001046FFF79DFA02E01046FFF7B0FAC2F3D8
:10F8C0000D0101EB4000184482E71046FFF790FA63
:10F8D0009FE71046FFF7A3FA9BE72DE9FE4FF84C90
:10F8E000FA4E4AF28428A06DDFF8D893F64F30F82C
:10F8F000022BA065018802F47F4343EA112C4FF6E6
:10F90000FF7303EA0125D3B223662B43B6F8785F71
:10F910000295B6F87C5F0195B6F8805F0095B6F861
:10F9200084EFACEB080204F16C05C44563D073DCD2
:10F9300048F28668ACEB0802C4456ED034DC48F26D
:10F940008A47ACEB07024FF00106BC456FD019DCCB
:10F9500048F28447ACEB0702BC4569D00DDC0CF5DE
:10F96000FF4CBCF5803C7BD0BCF5007F78D0ACF57B
:10F97000806CBCF1020C74D1C0E0022A72D0042A5F
:10F98000F9D1CFE0B2F5FB7F6DD006DC022A6BD057
:10F99000042A6AD0062AEED1DDE0B2F5FC7F7DD0E4
:10F9A000B2F5FD7FE7D1E6E0C84941F6FF18A2EBCA
:10F9B000080CB1F838BEB1F86CAFB1F8709FB1F86F
:10F9C000741F42456BD017DC41F6FC18A2EB080C03
:10F9D000424574D009DC022A72D002F20662B2F506
:10F9E000005218D0012AC6D1DEE0BCF1010F1DD0B3
:10F9F000BCF1020FBFD1F5E0BCF5FE7F7CD00DDC81
:10FA0000BCF1010F79D0BCF1020F28D0ACF5807C9D
:10FA1000BCF1FB0CAFD1BDE00BE0B1E0ACF5807CFC
:10FA2000BCF1FD0C4BD0BCF1010FA4D1D1E07EE0C4
:10FA30006AE04FF4FF78B2F5027F70D025DC40F227
:10FA40000127A2F20121BA426AD016DC424568D0F1
:10FA50000CDC012A23D0022A4FD0032A8BD1DFE00D
:10FA600044E077E055E07CE067E06CE0A2F580726E
:10FA7000FF3A6ED0012A8ED1F6E007296AD2DFE87C
:10FA800001F069F2F1F0EFEEED0040F2FF310026F7
:10FA9000A2F2FF3041F6322B8A4201E066E0ABE091
:10FAA00070D017DCB2F5037F6DD00ADCA2F50072CE
:10FAB000093A69D0012A68D0022A94D12FE17EE068
:10FAC00064E0A2F500720D3A78D0A2F58072F13AA6
:10FAD00089D13CE143F67E6C43F2AE6A0728CDD271
:10FAE000DFE800F038FAF9F8F7F6ED002B80801C1B
:10FAF000A065FFF772FC9DE056E087E0C8B2FFF713
:10FB000041F800F00F0029E0C8B2FFF73BF8C0B29F
:10FB100024E0C8B2FFF736F8C0F30B001EE0EBE0BC
:10FB2000A6E08BE0C8B2FFF72DF880B216E0C8B2AD
:10FB3000FFF728F8C0F3130010E0C8B2FFF722F86F
:10FB400020F07F400AE0C8B2FFF71CF820F07040B8
:10FB500004E077E02EE1C8B2FFF714F82860A6723F
:10FB600025E103EB0901D1F8001E02E003F1202397
:10FB7000196829601CE103EB0901D1F8001AF8E7C4
:10FB8000D959F6E7EBE0D5E0BAE0C4E0D919D1F8ED
:10FB9000D017EEE70BEB03012980801CA065FFF76F
:10FBA0001CFCB6F83A1E44E00AEB03012980801CD5
:10FBB000A065FFF712FCB6F86E1F3AE0BEE009EB55
:10FBC00003012980801CA065FFF707FCB6F8721FAF
:10FBD0002FE019442980801CA065FFF7FEFBB6F8D2
:10FBE000761F26E00299801C19442980A065FFF742
:10FBF000F4FBB6F87A1F1CE00199801C1944298097
:10FC0000A065FFF7EAFBB6F87E1F12E00099801CA2
:10FC100019442980A065FFF7E0FBB6F8821F08E0D1
:10FC20000EEB03012980801CA065FFF7D6FBB6F818
:10FC3000861F08446880A06D001FBAE01846FFF7D1
:10FC400005F902E01846FFF722F92066C3F3052004
:10FC5000FEF798FF00F00F002860A8E041E03CE0CC
:10FC600023E01EE012E00DE01846FFF7EFF802E097
:10FC70001846FFF70CF92066C3F30520FEF782FF54
:10FC8000C0B2E9E71846FFF7E1F802E01846FFF7CF
:10FC9000FEF82066C3F30520FEF774FFC0F30B00E7
:10FCA000DAE71846FFF7D2F802E01846FFF7EFF858
:10FCB0002066C3F30520FEF765FF80B2CCE790E035
:10FCC0003000002000100020003000200010002034
:10FCD00083E077E061E055E04CE01846FFF7B6F8C6
:10FCE00002E01846FFF7D3F82066C3F30520FEF7BD
:10FCF00049FFC0F31300AFE71846FFF7A7F802E08B
:10FD00001846FFF7C4F82066C3F30520FEF73AFF54
:10FD100020F07F40A0E71846FFF798F802E0184669
:10FD2000FFF7B5F82066C3F30520FEF72BFF20F0A0
:10FD3000704091E71846FFF789F802E01846FFF790
:10FD4000A6F82066C3F30520FEF71CFF84E71846DB
:10FD5000FFF77CF806E000BF00F1202030E01846F5
:10FD6000FFF795F8C3F30D0101EB400080B2404569
:10FD700041D2F1E71846FFF769F806E04844D0F8A9
:10FD8000000A69E71846FFF782F8C3F30D0101EB9B
:10FD9000400080B240452ED2F0E71846FFF756F8F3
:10FDA00013E0594640F64370FEF723FC2E60A06D29
:10FDB000801CA065A06D001DA065286892E43844F1
:10FDC000006849E71846FFF762F8C3F30D0101EB3D
:10FDD000400080B26045F2D3E3E71846FFF736F8FB
:10FDE00002E01846FFF753F8C3F30D0101EB4000A2
:10FDF00080B2504506D3594640F64370FEF7F9FBF2
:10FE00002E60D7E73844D0F8D00725E72DE9F04138
:10FE1000FE4D4FF6FF77AC6D34F8020B34F8022B31
:10FE200000F47F4114F8023B41EA1221AC6507EA75
:10FE300002222688C0B2104307EA0626DAB232430D
:10FE400005F16C031E1FA1F50047803F1AD0A1F5F4
:10FE50000247803F16D0EE4AA1F50643803B17D0FB
:10FE6000A1F50643823B17D0A1F50643843B16D08B
:10FE7000E84AA1F50643863B15D0A1F50643883B29
:10FE800014D019E018805A80186803F0CBFD10E0F8
:10FE90001044D0F8000E0CE000F1202004E01044E3
:10FEA000D0F8000A05E01044006802E01044D0F8E1
:10FEB000D007A41C3060AC653068BDE8F0812DE946
:10FEC000F05FD2484179C90751D0FEF7A6FE04463B
:10FED000FEF7A3FE8346FEF7A0FE8246FFF77DFAFB
:10FEE0001FFA80FC0023DFF83093C94A3BE000BFD3
:10FEF0000BEB030002EBD00100F007070E7819F8B6
:10FF00000770C3EBC3053E430E70002155446018D3
:10FF100002EBD00600F00707367819F807703E426A
:10FF20000DD06F1802EBD70607F0070796F8008090
:10FF300019F8070048EA000886F800800DE0681804
:10FF400002EBD006DFF8D08200F0070008F10808C5
:10FF5000377818F8000007403770491CC9B20729E4
:10FF6000D5D95B1CDBB26345C2D3BDE8F09F816D80
:10FF700010318165F9E72DE9F041A44C6079C007A3
:10FF800032D0FFF72AFA6066FFF7AEF8FFF725FADE
:10FF90000746A06D4FF6FF76001F0125A06515E00E
:10FFA000A07A01281AD006EA45002082A06D083800
:10FFB000A065FFF712FA6066607A012811D006EAA0
:10FFC00045002082FFF790F86D1C2DB2BD42E7DBA3
:10FFD000A06D001DA065002020826EE706EA0510D6
:10FFE000E3E706EA0510ECE7A06D0C30A06564E7D6
:10FFF0002DE9FF5FDFF8148298F80500C0075FD095
:020000040801F1
:10000000FEF70BFE854D35F8107005EB4000468875
:10001000B0F804A0FEF701FE35F8101005EB400023
:100020000091B0F802B0B0F80490FEF7F6FD044677
:10003000FEF7F3FDFF22DFF8D8E188F800200EEB91
:10004000D001DFF8D4810A7800F0070308F108082E
:10005000039318F803301A400A70431C0EEBD302C6
:1000600003F0070392F800C0029318F80330801CD5
:100070000CEA030C82F800C00EEBD00C00F0070075
:100080009CF80030019018F80000E64603408CF818
:10009000003035F81450DFF880C1BD4212D85F48F7
:1000A00000EB4400B0F80280B0450BD8B0F80480F3
:1000B000D04507D2039A08781CF802201043087034
:1000C000BDE8FF9F5548BD4215D300EB4407798832
:1000D000B14210D351450ED3009EB5420BD85945BD
:1000E00009D8BE884E4506D8029811781CF8000041
:1000F00001431170E4E700998D42E1D300EB440025
:1001000042885A45DCD381884945D9D901981CF8E1
:10011000000003438EF80030D2E72DE9FC5F3B4D31
:100120003D4F3B4C6879C00752D0FFF76FFE0190FE
:10013000FFF76CFE0090FFF769FE8346FEF76DFD4A
:10014000FF21297004EBD00600F0070A07F108022E
:10015000317812F80A3019403170411C04EBD10596
:1001600001F007092B7812F80910801C0B402B7046
:1001700004EBD00400F00708217812F808000140D1
:1001800021705946019803F060FD06D2317817F8C6
:100190000A0001433170BDE8FC9F5946019803F005
:1001A00059FC0AD85846009903F054FC05D8287821
:1001B00017F8091008432870EDE75946009803F036
:1001C00049FCE8D2207817F8081008432070E2E7CD
:1001D000A86D2030A865DEE72DE9F0470B4E707959
:1001E000C00762D0FFF779FB8246FFF776FB054632
:1001F000FFF773FB0446FEF710FDFF213170C117B6
:10020000034E00EB517206EBE20309E030000020E0
:100210000010002000300020EC5F000800100020DB
:1002200022F00702F94FA0EB0209197819F807200C
:1002300011401970411CCA1701EB527806EBE80215
:1002400028F00708A1EB080892F800C018F807107A
:100250000CEA010C811C82F800C04FEAE17C01EB42
:100260005C7C06EBEC012CF0070C801CA0EB0C0076
:100270000E78C75D3E40E54F0E70083FA24506DD93
:10028000187819F8071008431870BDE8F087AC42D9
:1002900005DC107818F8071008431070F5E7A54240
:1002A000F3DAC05D06430E70EFE7B06D2030B06545
:1002B000EBE72DE9F047D64E7079C0075BD0FFF72A
:1002C0008CF88246FFF789F80546FFF786F8044662
:1002D000FEF7A3FC01B2FF203070C817CD4E01EB32
:1002E000507206EBE20322F00702C84FA1EB0209AD
:1002F000187819F8072010401870481CC21700EB36
:10030000527806EBE8004A1C28F00708A2EB080820
:1003100090F800C018F807200CEA020C8A1C80F83C
:1003200000C04FEAE27C02EB5C7C06EBEC022CF0B6
:10033000070C891CA1EB0C011678CF5DDFF8CCC24D
:100340003E401670ACF1080CA24505DD187819F88E
:100350000C100843187098E7AC4205DC017818F8D7
:100360000C201143017090E7A5428EDA11F80C00C1
:100370000643167089E7B06D1030B06585E72DE94A
:10038000FC5FDFF88C8298F80500C00777D0FFF794
:1003900024F887B2FFF721F886B2FFF71EF885B27E
:1003A000FEF73BFC0446FEF738FCFF22DFF86492C0
:1003B00088F8002009EBD002DFF85082117800F0B5
:1003C0000703019318F8033019401170411C09EB21
:1003D000D10301F0070193F800C0009118F8011053
:1003E000801C0CEA010C83F800C009EBD00100F07E
:1003F000070E91F800C018F80E0089460CEA000CB0
:1004000081F800C08449E346A8F1080C31F81400D3
:10041000B84210D801EB440ABAF80280B0450AD8B5
:10042000BAF80480A84506D2019910781CF801108A
:1004300008431070AFE6B8420FD101EB4402B2F8A6
:100440000280B04509D19288AA4206D10099187855
:100450001CF80110084318709DE6B842EAD301EB7E
:1004600044004188B142E5D38088A842E2D91CF813
:100470000E104BEA010089F800008CE6FFE7D8F87F
:1004800058101431C8F8581085E62DE9F05F604C1B
:10049000DFF878815F4D6079A8F10808C0075CD06B
:1004A000FFF7B4FCE062FFF7B1FC2063FEF7B5FB99
:1004B00001B2FF202070C81701EB507005EBE00778
:1004C00020F00700514AA1EB000B3B781BF802001B
:1004D00003403B70481CC31700EB537305EBE30666
:1004E00023F00703A0EB030A96F800C01AF80200F5
:1004F0000CEA000C881CC31700EB537005EBE005F9
:1005000020F00700891C86F800C0A1EB00092B78B9
:1005100019F8020003402B70D4E90B0103F095FB9E
:1005200005D238781BF80810084338701DE5D4E967
:100530000B0103F023FA05D130781AF808100843AC
:10054000307012E5D4E90B0103F084FAEED228787A
:1005500019F808100843287007E5A06D1830A06549
:1005600003E52DE9F0412A4C6079C0075BD0FFF725
:10057000B4F96063FFF7B1F9A063FEF74EFBFF210A
:1005800000B22170C11700EB517522491F4E01EBDB
:10059000E50325F00705A0EB050E1A781EF80650B6
:1005A0002A401A70421CD51702EB557C01EBEC0275
:1005B000451C2CF0070CA5EB0C0C17781CF806500A
:1005C0002F40851C1770EF1705EB577701EBE701FC
:1005D00027F00707801CC01B0D78865D35400D7025
:1005E000D4E90D67094C083CBE4206DD18781EF8B8
:1005F000041040EA010018705FE40FD110781CF875
:10060000041040EA0100107057E40000F45F000895
:10061000300000200010002000100020005D45EA9E
:1006200000050D7049E4A06D00F11800A06544E4D8
:100630002DE9F041FDF7A3FFFE4CE8B3FFF74DF9BC
:10064000E063FFF74AF92064FEF7E7FAFF2100B202
:100650002170C11700EB5175F749F84E01EBE50326
:1006600025F00705A0EB050E1A781EF806502A4063
:100670001A70421CD51702EB557C01EBEC02451CAD
:100680002CF0070CA5EB0C0C17781CF806502F402B
:10069000851C1770EF1705EB577701EBE70127F083
:1006A0000707801CC01B0D78865D35400D70D4E9AE
:1006B0000F67E24C083C00E015E0BE4206DD18780A
:1006C0001EF8041040EA0100187086E406D1107884
:1006D0001CF8041040EA010010707EE4005D45EA59
:1006E00000050D7079E4A06D00F11800A06574E4B8
:1006F0002DE9F047CF4C6079C00757D0FEF76DFE6B
:100700008146FEF76AFE8046FEF787FAFF2100B2B7
:100710002170C11700EB5174C749C84D01EBE403C8
:1007200024F00704071B1A787C5D00F1010C2240BD
:100730001A70421CD41702EB547601EBE60226F045
:100740000706ACEB0606147816F805C004EA0C049C
:100750001470841C4FEAE47C04EB5C7C01EBEC013C
:100760002CF0070C801CA0EB0C0C0C781CF805007E
:1007700045460440DFF8C4820C70A8F10808A9457A
:1007800006DD187817F8081040EA010018707CE5BB
:1007900006D1107816F8081040EA0100107074E5D0
:1007A0001CF8080044EA00040C706EE5A06D00F12E
:1007B0000C00A06569E52DE9F047FDF7E0FE9D4CD2
:1007C000E8B3FEF70AFE8146FEF707FE8046FEF715
:1007D00024FAFF2100B22170C11700EB5174964931
:1007E000964D01EBE40324F00704071B1A787C5DA7
:1007F00000F1010C22401A70421CD41702EB54760F
:1008000001EBE60226F00706ACEB0606147816F8B4
:1008100005C004EA0C041470841C4FEAE47C04EB69
:100820005C7C01EBEC012CF0070C801CA0EB0C0CA9
:100830000C781CF80500454604400C7000E01AE0F6
:10084000DFF8F881A945A8F1080806DD187817F83F
:10085000081040EA0100187017E506D1107816F864
:10086000081040EA010010700FE51CF8080044EA87
:1008700000040C7009E5A06D00F10C00A06504E512
:1008800070B56C4C6E4DA06D2844C0F34F0001F064
:10089000D9FE002860796B494FEAC07001D0F0B1F1
:1008A0002EE068B3A06D42195010C31700EB5370CF
:1008B00001EBE00120F00700C0EB62005F4A0B781B
:1008C000083A805C03430B70FFF707F8A16D083905
:1008D000801CA1656066BDE87040FEF7FBBAA06DA4
:1008E00042195010C31700EB537001EBE00120F0E8
:1008F0000700C0EB6200514A0B78805C03400B702C
:10090000A06D0830A06570BD2DE9F047494E7079A3
:10091000C00751D0FEF79FF98146B06DB046001D6B
:100920003746B065FEF759FD86B239780020FF29B9
:100930000CD0D8F858101FFA89F508390446012759
:10094000A1464FF6FF7AC8F8581021E0002007E0D2
:1009500039F9102000F10100551944EBE27480B21E
:10096000B042F5D3D8F858100839C8F8581014E038
:10097000D8F85810091FC8F858100AEA0711A8F843
:100980001010FEF768F9451949EB04047F1CBFB24B
:10099000B742EDD3FF2188F80010324600232846E5
:1009A0002146F4F773F94446C8F86400FEF79CFB4F
:1009B000A06D001DA06568E4B06D0C30B06564E406
:1009C0002DE9F0471B494879C2070846806D7AD067
:1009D0008946C865FEF781FFC21700EB127121F04E
:1009E0000F03C51A0911CB1701EB137323F00F0383
:1009F000CE1A00EB12610912CB1701EB137323F02F
:100A00000F03CF1A00EB12510913CB1701EB13732D
:100A100000EB124023F00F030014A1EB030CC217EC
:100A200000EB127121F00F03C31A0911CC1701EB6F
:100A3000147409E03000002000100020F45F00086A
:100A4000A49FFFF7CD07002024F00F040C1B00EB40
:100A50001261091200EB125000134FEAE178C2173D
:100A600001EB187800EB127228F00F0822F00F0249
:100A7000A1EB0801801AFE4A504343F60952514344
:100A800000EB811040F635414C4340F271214B435D
:100A900000EB44100CEB4C0100EB0310C1EBCC114C
:100AA00000EBC10007EBC70101EB071100EB810070
:100AB00006EB860100EB41004119C9F86410BDE85E
:100AC000F047FEF707BA1030886544E470B5FEF7CA
:100AD00084FC0546FEF7A1F80446FEF77EFCE549D6
:100AE00001EB400131F8022C2A40002101E0491CB1
:100AF000C9B28142FBDBE0490120521E904021F83F
:100B0000140070BD2DE9FF47DA4DDFF87083903D8A
:100B1000DB4C6879DB4EC0074FF0000770D0FEF762
:100B20005CFC8146FEF759FCA96D11F8042BAA70F4
:100B3000A965D149B1F8181F814205DB94F8E3118A
:100B400041F0200184F8E311002A56D194F8F21103
:100B5000890752D4317800294FD114F8A01F41F0F1
:100B60000101217094F8431101F0DF0184F8431171
:100B700001213170C44904F24314088009EBC90013
:100B8000C249000191FBF0F54FF40070ADF80C0084
:100B900003208DF80E0010208DF80F0003A9BC482B
:100BA0006D1EF0F7D2F901210220F0F717FC46463E
:100BB0004046F0F7E1FC4720ADF80000ADF80450E6
:100BC000ADF80670ADF8027069463046F0F76CFD7E
:100BD00001213046F1F738FA012211463046F1F78B
:100BE00021F801213046F1F708F801210220F0F741
:100BF000F5FBE07B40F00800E073BDE8FF87FFE70E
:100C0000A86D017A00F10C0011F0FF01A970A86530
:100C1000F3D130780128F0D19E48F0F7EEFF0021A3
:100C200045464046F0F7E9FF01212846F1F70CFA66
:100C3000002201212846F0F7F5FF377014F8A00FC5
:100C400000F0FE00207094F8520100F0F70084F8E4
:100C50005201D2E72DE9F041864C8F4D903CA06DBA
:100C60002844C0F34F0001F0EDFC8C4ED0B1607908
:100C700040006071A06D008820F4504001F0F0FC4D
:100C8000A0BBA06D41194810C21700EB527206EBD1
:100C9000E20022F00702C2EB6101814A0378895C1D
:100CA0000B4022E07E4F207B083F012860794FEA0D
:100CB00040006071A06D008820F450401AD001F00F
:100CC000CFFC98B1607940F001006071A06D4119CE
:100CD0004810C21700EB527206EBE20022F0070246
:100CE000C2EB61010378C95D0B430370A06D801CEA
:100CF000A06581E401F0B4FC0028F7D0208C604AA4
:100D000002EBD00100F007000978385C0142EDD019
:100D1000607940F001006071A06D41194810C21760
:100D200000EB527006EBE00220F00700C0EB610020
:100D30001378C05D03431370D8E72DE9F0414D4CA3
:100D4000554D903CA06D2844C0F34F0001F07AFC53
:100D5000534F524E083F80B3207B012860794FEA01
:100D600040006071A06D008820F4504003D001F075
:100D700077FC18B354E001F073FCA0BB208C404A10
:100D800002EBD00100F007000978385C014247D03F
:100D9000607940F001006071A06D41194810C217E0
:100DA00000EB5272481022F0070106EBE203401AF2
:100DB0001D78C05D05431D7032E015E0607940F09C
:100DC00001006071A06D41194810C21700EB52700C
:100DD00006EBE00220F00700C0EB61003049137819
:100DE000405C03401BE01BE06079400000F0FE0027
:100DF0006071A06D008820F4504001F031FC78B1A2
:100E0000A06D41194810C21700EB527006EBE002CA
:100E100020F00700C0EB61001378C05D034313703E
:100E2000A06D801CA06550E42DE9F041114C1A4ED4
:100E3000903CA06D3044C0F34F0001F003FC00284B
:100E4000A06D164F008820F4504030D001F008FC0F
:100E500040BBA06D81194810C21700EB527007EB20
:100E6000E00220F00700C0EB610013780C491AE0A3
:100E700080969800C0000020001000200004004070
:100E800000100020F1000020F200002000A24A041F
:100E900000100140000C0040A49FFFF7CD07002088
:100EA000F45F000821E0405C034013701DE001F096
:100EB000D7FBD0B1A06D81194810C21700EB52705A
:100EC00007EBE00220F00700C0EB6100FA4913785D
:100ED000405C034313706079C10706D040F0010005
:100EE0006071A06D801CA06503E7607900F0FE00D2
:100EF000F6E72DE9F041F14CF14EA06D3044C0F31E
:100F00004F0001F09FFB0028A06DEE4F008820F4F9
:100F100050401ED001F0A4FB78BBA06D8119481091
:100F2000C21700EB527007EBE00220F00700C0EBA5
:100F30006100E14913780831405C03401370607927
:100F4000C1071AD040F001006071A06D801CA0653F
:100F5000CFE601F085FB80B1A06D81194810C21762
:100F600000EB527007EBE00220F00700C0EB6100DD
:100F7000D1491378405C03431370607900F0FE00A0
:100F8000E2E770B5CD4CCE4DA06D2844C0F34F00C4
:100F900001F058FB0028A06DCA4E008820F4504094
:100FA00015D001F05DFB38BBA06D41194810C21788
:100FB00000EB527006EBE00220F00700C0EB61008E
:100FC000BD4913780831405C0340137014E001F010
:100FD00047FB88B1A06D41194810C21700EB527051
:100FE00006EBE00220F00700C0EB6100B249137885
:100FF000405C0343137002E06079C00703D060795E
:1010000040F0010002E0607900F0FE006071A06D28
:10101000801CA06570BD70B5A84CA94DA06D28447A
:10102000C0F34F0001F00EFB0028A06DA54E008814
:1010300020F450401CD001F013FB90B9A06D411971
:101040004810C21700EB527006EBE00220F00700D8
:10105000C0EB6100984913780831405C034013707D
:1010600002E06079C00719D0607940F0010018E013
:1010700001F0F6FA0028F4D0A06D41194810C2170B
:1010800000EB527006EBE00220F00700C0EB6100BD
:1010900089491378405C03431370E2E7607920F0DC
:1010A00001006071A06D801CA06570BD834A802323
:1010B000916D891C91650988B3EB112F05D1824987
:1010C000400851F82000801C90657047F0B57B4CBB
:1010D0008023A26D921CA2651188B3EB112F19D148
:1010E0007A4D3E21A5F5017305EB410735F81160F6
:1010F0007E8053F8216003EB8107491E7E6011F06A
:10110000FF01F1D1617929806F4940081A6051F8D7
:101110002000A065F0BD10B5684CA06D008820F4DB
:101120005040FDF765FBA06D801CA06510BD10B59B
:10113000624CA06D008820F4504001F0B5FAA06D1B
:10114000801CA06510BD10B55C4CA06D008820F41B
:101150005040FDF703FBA06D801CA06510BD10B5CD
:10116000564CA06D008820F45040FDF758FAA06D51
:10117000801CA06510BD10B5504CA06D008820F4F7
:101180005040FDF770FAA06D801CA06510BD4B4B60
:1011900000B5986D008820F45040FDF789FA986DED
:1011A000801C986500BD10B5444CA06D008820F4EB
:1011B0005040FDF792FAA06D801CA06510BD10B5DF
:1011C0003E4CA06D008820F45040FDF79BFAA06DC6
:1011D000801CA06510BD10B5384CA06D008820F4AF
:1011E0005040FDF7A4FAA06D801CA06510BD2DE94C
:1011F000F007324A364F0125916DDFF8BC90DFF8D9
:10120000D4C011F8020B91650B78DFF8ACA000EBAD
:10121000032086B2D683107A09F10809030900F089
:101220000F04A54000F5606807EB430308F00704CE
:101230000CEBD80C03F59C63C8282AD38F78091DC2
:101240009165097806EB074606EB016189B2D18307
:10125000214AAEB202EB800215688D4204DA1B8887
:101260009E4301D06D1C15608D4205DA9CF800107C
:1012700019F80420114004E09CF800101AF804202A
:1012800011438CF80010BDE8F00700F51C50FDF785
:1012900065BA07EB400101F5206191640A88ADB29F
:1012A000B24204D21B889D4301D0521C0A8091B2E5
:1012B000B142E1D2DAE70000EC5F00083000002024
:1012C000A49FFFF7CD070020240100202C0500205B
:1012D0000010002000100020E01800202DE9F0038D
:1012E000DC49DB4E0127C88B334606EB400000F596
:1012F0000050DFF864830588CD83087AA8F10809D7
:10130000020903EB420300F00F04D44AA74000F5A2
:10131000606C0CF0070402EBDC0203F59C63C82848
:1013200027D306EB450606F500561FFA87FCB6786C
:1013300005EB0645CA4EADB206EB8006CD83376895
:10134000AF4205DA1B883CEA030C01D07F1C3760F2
:10135000CB6C1B88AB42137803D218F804402340AF
:1013600002E019F80440234313708A6D121D8A6548
:1013700019E006EB400606F52066CE643188BFB260
:10138000A94204D21B889F4301D0491C318089B2F5
:10139000A942117803D818F80430194002E019F86E
:1013A000043019431170BDE8F00300F51C50FDF73F
:1013B000D5B9F0B5A74AA84F916DA7F1080C11F85F
:1013C000020B91650B7800EB03201FFA80FEA2F858
:1013D0001EE0107AA14B00F5606603EBD60506F01F
:1013E00007042B78C82819D3091D916509780026B0
:1013F00006EB016189B2D183994A52F820208A42D2
:1014000002DA395D0B4002E01CF804100B432B702C
:10141000BDE8F04000F51C50FDF7A0B98C4901EB88
:10142000400101F52061116509887145ECD2E8E7BA
:10143000F0B58849864E0B46087ADB8B874A06EB67
:10144000430300F5606E03F5005302EBDE05824FA7
:101450001B882A78A7F1080C0EF00704C82818D3B7
:1014600006EB430606F50056B67803EB06437C4EC2
:101470009BB2CB8356F820609E4202DA3B5D1A4055
:1014800002E01CF804301A432A708A6D121D8A6526
:101490000FE006EB4006CB8306F520664E653188EB
:1014A000994202D2395D0A4002E01CF804100A4356
:1014B0002A70BDE8F04000F51C50FDF74FB92DE94A
:1014C000F041644C40F2011C2146A06D88260027A3
:1014D00030F8023B4979A3F2011204F16805634533
:1014E0007BD065DC3D2B79D023DCA3F102033B2BC1
:1014F00075D2DFE803F0F1F0EFF1F0EFEEED747488
:10150000ECEB74EAE974E874E774747474747474DA
:10151000EA74747474747474E6E5E4E3E2E1E0740C
:10152000DFDEDD74DCDBDAD9D8D7D6D5D4D3D2D19F
:10153000D000474E512B71D00FDCA3F13E03132B8B
:101540004DD2DFE803F0EBEAE9E8E7E6E5E4E3E2C1
:10155000E1E0DFDEDDDCDBDAD900762B77D014DCEE
:101560006A2B7FD008DC522B7DD0532B7CD0602B94
:101570007BD0622B33D1B8E3702B77D0712B76D030
:10158000722B75D0732B2AD1DFE3C02B71D008DC0E
:10159000782B6FD07A2B6ED0822B6DD0942B1ED1EE
:1015A000F7E3ED2B69D0EE2B68D0F12B17D1F1E3E7
:1015B000D42A64D064DC652A63D030DC352A61D05B
:1015C00017DC112A5FD00BDC022A5DD0042A5CD024
:1015D000062A5BD00E2A02D1FEE3FEE33FE259E089
:1015E000122A54D0142A53D0162A52D0182A51D174
:1015F000F4E3552A71D008DC362A6FD04F2A6ED01A
:10160000512A6DD0532A45D1E9E35B2A69D05D2A7E
:1016100068D0632A67D0642A3CD1F1E31CE3CB2A6B
:1016200062D07DDCC42A61D008DC662A5FD0C12A82
:101630005ED0C22A5DD0C32A2CD1F0E3C52A59D08E
:10164000C62A58D0C92A6AD0CA2A23D1E8E384E33B
:101650000010002030000020F45F0008001000207F
:10166000E018002046E301E312E31BE347E352E303
:101670005EE39CE37CE380E38FE39DE3A1E3F6E399
:1016800057E0F5E3F5E3F5E3BBE3DAE3CAE3F3E3BD
:10169000F3E3F3E38DE0D2E1C6E1BAE1AEE1A3E129
:1016A0009AE194E18EE188E176E16AE164E15EE14C
:1016B00058E14FE13EE138E116E10FE109E103E1D4
:1016C000F8E0EDE0D2E0BDE0A7E09BE0A0E08CE038
:1016D00086E080E07BE076E071E0F5E3F5E3F5E3BA
:1016E000F5E3F5E3F5E3F5E3F5E319E0F4E3F4E31B
:1016F000F4E3F4E3F4E3F4E3A1E28EE27BE270E2EC
:1017000060E256E247E23CE231E226E218E20DE214
:1017100002E2F3E1E5E1D6E1C4E1BEE1A4E1FAE3EE
:10172000CC3A082A45D2DFE802F0ECEBEAE9E8E738
:10173000E6E5F02A7CD012DCA2F1D702192A38D2D1
:10174000DFE802F0F2F1F0EFEEED3737ECEBEAE92B
:10175000E8E73737E6E5E4E3E2E13737E000FC2A83
:1017600067D00BDCA2F1F1020B2A22D2DFE802F0F3
:10177000F161F0EF2121EEEDECEBEA0040F63F7372
:10178000A2F63F719A426FD00ADCA2F570620F3A5E
:1017900050D0022A61D0142A67D0152A09D18EE0D0
:1017A00001297AD0022979D0A1F2BF71B1F5604F39
:1017B00075D0022140F64170FCF71BFF1FE0A065C9
:1017C000BDE8F041BFE4A065BDE8F041A3E4A06539
:1017D000BDE8F041ABE4A065BDE8F041FDF794B889
:1017E000A065BDE8F041FDF7EEB8A0650088010AEC
:1017F000862909D08E2905D1C0B200F098FFA06DCE
:10180000801CA065BDE8F081C0B200F05CFFF6E787
:10181000A065BDE8F04100F0AFBFA065C90710D0DA
:101820000088B6EB102FEDD1BDE8F041C0B23DE429
:10183000FEE3FEE3A065FCF7A2FE08B1A06DEFE7B2
:10184000A06D23E2A065C907FBD00088B6EB102F7E
:10185000D8D1BDE8F041C0B238E4A065FCF78FFEF6
:101860000028EDD0A06DF0E720E11EE0F94AA2F5D6
:101870000171107860710868A0653E2002EB40039A
:101880005B8822F8103001EB80035B6841F8203060
:10189000401E10F0FF00F1D1B4E71DE128E1FDE3A7
:1018A000A065BDE8F041FEF723BFA065BDE8F041AB
:1018B000FEF781BFA065BDE8F041FEF752BEA0650E
:1018C000BDE8F041FEF7B4BEA065BDE8F041FEF70B
:1018D000F0BCA065BDE8F041FEF77EBCA065C9077D
:1018E0007ED0FDF77AFD2BE0A065C90779D0FDF722
:1018F000F4FF35E0B2E3ACE3A6E3A0E397E391E3C2
:101900008BE385E3DBE3F2E3F2E3F2E3F2E3F2E31A
:10191000F2E3F2E3F2E3F2E3E2E3D7E3C8E3C2E3A4
:10192000BAE3B4E3AEE3A8E3A2E3A065BDE8F04107
:1019300001F02BB8A065C907D2D0FDF74EFDC0431A
:10194000606632E1F7E3F7E3F7E3F7E3F7E3F7E3A2
:10195000F7E3F7E3A065C907C8D0FDF7BEFFC043B2
:101960006066D5E0A065BDE8F041FEF704BBA06568
:10197000BDE8F04100F0D8BFA065BDE8F04100F03F
:10198000A6BFA065C907ABD0FDF727FD0546FDF74B
:1019900024FDA16D08390AE0A065C8073FF47CAFBB
:1019A000FDF79BFF0546FDF798FFA16D1039A16576
:1019B0006066FDF78FFA6566AAE0A065BDE8F041B4
:1019C00001F045B9A065BDE8F04101F0E4B8A065BB
:1019D000BDE8F04101F06AB9A065BDE8F04101E061
:1019E000EEE01EE2FEF7ECBFA065C90772D0FDF77E
:1019F000F4FC0546FDF7F1FC2844A1E7A065C90702
:101A000069D0E065FDF769FF0546FDF766FF2844EC
:101A1000A6E7A065C9075DD0E065FDF7DEFC0546D9
:101A2000FDF7DBFC281A8BE7A065C907E8D0E06565
:101A3000FDF753FF0546FDF750FF281A90E7A06514
:101A4000C90747D0E065FDF7C8FC0446FDF7C5FCB3
:101A50000546FDF700F904FB05F10160D2E6A0653B
:101A6000BDE8F04101F04BB9A065C90773D0E0654E
:101A7000FDF7B3FC0446FDF7B0FC0546FDF7CDF8D5
:101A800002B294FBF5F026F8120094FBF5F005FB8A
:101A9000104006EB42014880B4E6A065BDE8F04185
:101AA00001F054B9A065C90706D1EFE0A065FCF7C5
:101AB00066FD00283FF4C4AEFDF78FFCA16D091F41
:101AC000401CA1653CE7A065C90779D0FDF705FF7B
:101AD000401C19E03FE09FE0A065BDE8F041FEF743
:101AE000CFBEA065C9076CD0FDF777FC401E58E05B
:101AF000A065FCF744FD0028F6D1A1E6A065C90762
:101B0000E3D0FDF7EAFE401E6066A06D0838A065D0
:101B1000BDE8F041FDF7DEB9A065C9071BD0FDF7B0
:101B20005CFC0546FDF759FC054012E0A065C907BD
:101B300072D0FDF7D2FE0546FDF7CFFE05403AE72D
:101B4000A065C90707D0FDF748FC0546FDF745FC31
:101B50000543656629E00C3053E6A065C9075BD0F4
:101B6000FDF7BBFE0546FDF7B8FE054323E7A0657C
:101B7000C907F0D0FDF731FC0546FDF72EFC4540C6
:101B8000E7E7A065C90747D0FDF7A7FE0546FDF7C3
:101B9000A4FE45400FE7A065C90777D0FDF71DFCFF
:101BA00040426066A06D001FA065BDE8F041FDF7F2
:101BB0009BBAA065C90788D0FDF78FFE4042A3E716
:101BC000B5E063E0A065C9079AD0FDF706FC85B2D1
:101BD000FDF703FC80B225FA00F1C0F1100085404A
:101BE00017E0A065C8073FF457AEFDF776FE05463F
:101BF000FDF773FE1AE0A065C907DCD0FDF7EDFB29
:101C000085B2FDF7EAFB80B205FA00F1C0F11000E1
:101C1000C5402943616633E011E1A065C807E2D001
:101C2000FDF75BFE0546FDF758FE4042C54165667F
:101C3000A06D1038A065FDF74DF9A06DAFE1A0656E
:101C4000C90774D0FDF7C9FB85B2FDF7C6FBC540D7
:101C500015E000002C050020A065C807C3D0FDF7E3
:101C60003CFE0546FDF739FEC540E0E7A065C90723
:101C70005DD0FDF7B2FB85B2FDF7AFFB8540656631
:101C8000A06D0838A065FDF72FFAD9E5001DB8E56D
:101C9000A065C807A7D0FDF720FE0546FDF71DFE8D
:101CA0008540C4E7A065C90741D0FCF7B6FF0546EB
:101CB000FCF7B3FF217861B114E000BF02EBD5015E
:101CC00005F007060C789E5D34406D1C0C70ADB2BB
:101CD00001E0FB4AFB4B8542F0D993E526F81570ED
:101CE0006D1CADB28542F9D98CE5A065BDE8F04127
:101CF000FEF7ECBEA065BDE8F041FEF705BEA065AD
:101D0000C807EAD0FDF769FBF4F7B1F8F3F74CF92F
:101D1000F4F780F841E1A065C807DED0FDF7DDFDEE
:101D2000F4F7A5F8F3F740F9F4F774F808E675E06E
:101D3000A065C90772D0FDF750FB01F073FE286063
:101D400000F048FDA06D001F5BE5A065C90768D0E5
:101D5000FDF7C3FD01F066FECFE0DB4DA065C907CE
:101D600003D0FDF73AFB28704CE50A2129708DE776
:101D7000A065BDE8F041FEF7A2B8A065FDF7ADFD96
:101D80000546FDF7AAFDA84202D16079C10772D1CC
:101D900011E207E01AE0607134E5A065BDE8F041AA
:101DA000FEF7B0BEA065BDE8F04100F065BEA065DD
:101DB000BDE8F04100F020BDA065BDE8F041FEF7B0
:101DC00064BBA065BDE8F041FEF7A7B9A065C907EF
:101DD00027D0FEF71BF803E03FE005E082E0AEE02D
:101DE00001F000FE606689E0A065C90727D0FEF714
:101DF0000DF80446FEF70AF8214601F09BFC7CE052
:101E0000BCE0A065C9071AD0FEF700F80446FDF74C
:101E1000FDFF0146204601F049FF6EE09EE0D4E060
:101E2000ECE09AE0A065C90709D0FDF7EFFF044692
:101E3000FDF7ECFF0146204601F0DEFC5DE01830C6
:101E4000DFE4A065C907FAD0FDF7E0FF0446FDF71F
:101E5000DDFF214601F032FE4FE0A065C9077CD0CE
:101E6000FDF7D4FFF4F786F8F3F79EF843E0FAE0C5
:101E70008CE047E003E0A2E10AE011E01AE0A0658F
:101E8000C9076BD0FDF7C2FF01F0ACFD80B288E658
:101E9000A065C90761D0FDF7B9FF01F0A3FD5FE5BB
:101EA000A065C90759D0FDF7B1FFF4F763F8F3F760
:101EB000C5FC20E0A065C9077BD0FDF7A7FFF4F7BC
:101EC00059F8F3F76DFC16E03EE025E02DE031E037
:101ED0003FE046E04AE096E07CE062E06BE06FE0E5
:101EE0007DE081E0A065C90763D0FDF78FFFF4F7BF
:101EF00041F8F3F7F3FCF3F723FD2860BDE8F04168
:101F000000F068BCA065C90749D0FDF766FA011268
:101F100041EA002045E66CE0A065C8073FF4BCAC90
:101F2000FDF7DBFC4FEA3040EEE5A065BDE8F0418F
:101F3000FEF725BAA065BDE8F041FEF759B8A065E7
:101F4000BDE8F04100F074BDA065BDE8F04100F0CF
:101F5000FEBDA065BDE8F04101E02AE01FE000F011
:101F6000B7BDA065BDE8F04100F0D7BDA065C907C9
:101F700015D0FDF732FAFCF7E4FA0EE0A065C907C8
:101F800017D0FDF72AFAFCF7DCFAE9E4A065C907E7
:101F900005D0FDF722FAFCF7E3FA80B2D0E408306E
:101FA0002FE4A065C90704D0FDF717FAFCF7D8FAAB
:101FB000D6E4103025E4A065BDE8F041FFF7CFB8C6
:101FC000A065BDE8F041FFF7D6B8A065BDE8F041D7
:101FD000FFF7DDB8A065BDE8F041FFF7E4B8A06504
:101FE000BDE8F041FFF7EBB8A065BDE8F041FFF7B1
:101FF000F2B8A065BDE8F041FEF72CBEA065BDE8D3
:10200000F041FEF79ABEA065BDE8F041FEF70CBFB7
:10201000A065BDE8F041FEF76CBFA065BDE8F041EA
:10202000FEF7AFBFA065BDE8F041FEF7F4BF01E0E9
:10203000D3E01EE1A065BDE8F04100F0D9BEA06587
:10204000BDE8F04100F0AFBEA065BDE8F04100F092
:1020500019BFA065BDE8F04100F0EFBEA065BDE886
:10206000F04100F066BFA065BDE8F04100F03DBF63
:10207000A065BDE8F04101F034B8A065BDE8F041CD
:1020800001F00BB8A065BDE8F04100F09ABFA06573
:10209000BDE8F04100F071BFA06500E0F3E0BDE8ED
:1020A000F04100F0D6BFA065BDE8F04100F0ADBF43
:1020B000A065FDF792F90546FDF78FF90CE081E088
:1020C00000100020F45F0008F0000020A065FDF77C
:1020D00004FC0546FDF701FC85423FF456AE6AE07C
:1020E000A065FDF77AF90546FDF777F90EE059E0AE
:1020F00051E046E038E02DE025E012E00AE0FFE79D
:10210000A065FDF7EAFB0546FDF7E7FB85423FF7D3
:102110003CAE50E0A065FDF760F90546FDF75DF9BE
:1021200005E0A065FDF7D9FB0546FDF7D6FB854226
:10213000FFF62BAE3FE092E088E080E076E06EE0D4
:1021400064E05CE052E0A065FDF747F90546FDF765
:1021500044F905E0A065FDF7C0FB0546FDF7BDFBB2
:1021600085427FF412AE26E0A065FDF736F90546FC
:10217000FDF733F9854202DC6079C1071FD1607930
:102180007EE0A065FDF7A9FB0546FDF7A6FB8542AD
:102190007FF7FBAD0FE0A065FDF71FF90546FDF7E2
:1021A0001CF905E0A065FDF798FB0546FDF795FBDA
:1021B0008542BFF6EAAD607920F00100EBE540F022
:1021C0000100E8E5A065FDF708F90546FDF705F90A
:1021D00009E06079C1074AD152E0A065FDF77DFBB7
:1021E0000546FDF77AFB854241D0F2E7A065FDF791
:1021F000F4F80546FDF7F1F8854238DCE9E7A0651B
:10220000FDF7EBF80546FDF7E8F805E0A065FDF7FA
:1022100064FB0546FDF761FB854228DBD9E7A06535
:10222000FDF7DBF80546FDF7D8F805E0A065FDF7FA
:1022300054FB0546FDF751FB854218D1C9E7A0655F
:10224000FDF7CBF80546FDF7C8F805E0A065FDF7FA
:1022500044FB0546FDF741FB854208DDB9E7A06573
:10226000FDF7BBF80546FDF7B8F88542B1DB6079AC
:10227000A5E7A065FDF731FB0546FDF72EFBF4E76A
:1022800000F0FE0087E5A065277305E470B5FB4A02
:10229000F9480021FA4EB02443F67F659065038823
:1022A000B4EB132F02D1DBB246F82300491C89B2EC
:1022B000801CA942F3D3906570BDF2480021A0F8BC
:1022C000A210A0F8A0107047EB49EC4A10B5891E87
:1022D000002043F67E639165401C31F8024F80B2C6
:1022E0000F2C01D09842F7D3916510BD2DE9F0472E
:1022F000E548D0F83401DFF894C3DFF89493E54A59
:10230000E54BDE4C0127DF4E0025002847D0207921
:102310000921012814D093F8E001092813D000F016
:10232000FE0040F0020083F8E001A6F8185EE572B6
:10233000E570C2F8A0719CF80000002830D05DE183
:10234000257183F8E01198468A46C2F8A051E07AD8
:1023500058B9FFF79BFFE772FFF7B6FF43F67E61C0
:10236000884202D988F8E0A12EE1E07838B998F8DF
:10237000E01101F0F70141F0040188F8E011BE48D6
:10238000A0659CF8000008B9F0F7D8FDA16D088899
:10239000020A5E2A72D035DC5E2A70D201E030E19A
:1023A00026E1DFE802F0EF6C6C6C6C6C996C6C6C85
:1023B0006C6C6C6CB26C6C6C6C6C6C6C6C6C6C6C17
:1023C0006C6C6C6C6C6CC9C9C9C9C9C9C9C9C9C9AB
:1023D000C9C9C9C9C9C9CECECECECECECECECECE3B
:1023E000CECECECECECED3D3D3D3D3D3D3D3D3D3DB
:1023F000D3D3D3D3D3D3D9D9D9D9D9D9D9D9D9D971
:10240000D9D9D9D97F2A71D015DCA2F15F02202A4F
:1024100035D2DFE802F0A1A6A6A6A6A6A6A6A6A685
:10242000A6A6A6A6A6A6A6ADADADADADADADADAD0D
:10243000ADADADADADADDC2A1FD028DCCC2A0BD0C4
:1024400012DCC82A08D008DCB02A6ED0C52A03D016
:10245000C62A01D0C72A12D18FE0C92A03D0CA2ABE
:1024600001D0CB2A0BD188E0D82A06D008DCCD2AAF
:1024700071D0CF2A6FD0D52A01D184E06CE075E00D
:10248000D92A03D0DA2A7ED0DB2A6FD17BE0EC2A6E
:102490007ED010DCE82A7BD006DCDD2A73D0DF2A70
:1024A00071D0E52A62D173E0E92A71D0EA2A6FD0AF
:1024B000EB2A5BD16CE0F12A6FD006DCED2A67D005
:1024C000EF2A65D0F02A7CD167E0F22A65D0F32AA2
:1024D00063D0FF2A75D165E0E071891CA165088889
:1024E000000A802803D086285FD10BE040E06079A5
:1024F000C00702D000F019FE57E0891CA16500F06A
:102500002FFE52E000F03DFE4FE02072891CA165D5
:102510000888000A802802D0862846D109E0607920
:10252000C00703D0FEF763FE3FE042E0FEF741FF45
:102530003BE000F05DFE38E0C0F30B00FCF76FF805
:1025400033E0C0F30B00FCF78EF82EE0C0F30B0075
:10255000FCF7AEF829E010E0C0F30B00FCF7BDF883
:1025600023E0C0F30B00FCF7CDF81EE029E00AE001
:10257000C0F30B00FCF7DBF817E0C0F30B00FCF72F
:10258000EDF812E018E0C0F30B00FCF731F90CE0B5
:10259000C0F30B0000F088F807E0C0F30B00FCF775
:1025A00068F902E0C0B2FCF77CF9A06D801CA06560
:1025B000ECE6891CA165E9E6C0B21C2804D00F280E
:1025C00002D0FEF77CFFE1E6B9F80010A6F8181E6D
:1025D000A6F8161EA6F8141EA9F80050E77098F881
:1025E000E01101F0FB0141F0080188F8E01125E05D
:1025F000FFF763FEF0F7A2FCF0F7FDFD25736573AE
:102600001CE0FFF75AFE93F8E00100F0FE0040F0F6
:10261000020083F8E001A6F8185EE572E570C2F8E2
:10262000A0718CF80050F0F789FC25736573207950
:1026300020B92771A9F80050F0F7DDFDA6F8025E79
:10264000BDE8F0871549164A01EBD00100F00700FC
:102650000978105C014201D00120704700207047CA
:102660000D4A02EBD0010E4A00F007000978105C19
:10267000014217D0012070475C6000083000002044
:10268000240100200010002000002242F50000205C
:10269000E40000200080214200100020CD0700202F
:1026A000EC5F00080020E6E7FE494979C907E2D05F
:1026B000FD49FE4B01EBD00100F007000A78185CE1
:1026C00002400A70D7E7F0B5F649F74AF74D497965
:1026D000CB0700F50C5101F0070402EBD10121D02A
:1026E00000F5C06302EBD30603F007033778EB5C19
:1026F0001F4000F5185302EBD302377003F00703B5
:102700001678EB5C1E401670A5F108030A781B5D75
:102710001A430A70E64A002102EB400000F580509F
:102720000180F0BD08782A5D10400870F0BDF0B45B
:10273000DC4B5979C9071AD0DD49DFF86CC300F1C9
:10274000E002A0F1C807002401EB400102F00705F8
:10275000D64E0CEBD20201F52061372F01D821F8BB
:10276000024B59620C801178735D19401170F0BCF6
:1027700000F55C50FBF7F2BFCA4910B44879C207B4
:102780000846806D23D010F8022B8865008800234E
:10279000010AC74C86290AD0882908D080290BD085
:1027A00010BC41F6651140F64170FBF722BF02EB09
:1027B0000020C0B2002103E002EB0020C0B2E821FB
:1027C00001EB5000C0B224F8103010BC7047001D5F
:1027D0008865FAE710B5FCF720FAB249B44A6831C7
:1027E0000B8822F8103002EB400049884180AD4848
:1027F000816D091D816510BD2DE9F047A94840791B
:10280000C00763D0FCF727FAB0F80090FCF723FA72
:10281000B0F900A0FCF71FFA0446FCF71CFAB4F963
:102820000050B4F90860B4F9188095FBF6FCB4F9CF
:102830000E60E7880CFB068CB4F81080B4F90A30FF
:10284000B4F90C20A6EB080666447E43A683678A8B
:1028500004F10E01A7EB0906E681B4F90440B1F9D1
:102860000660C4F10107664307FB0A6403FB0255D7
:1028700092FBF5F624B28C805343B1F9087093FBB8
:10288000F5F23C44B1F90670B1F90C307F4204EB2B
:102890004704664302FB03624A81B0F90020B1F9A4
:1028A0000E301A4447F6FE739A4201DD5A1C04E0CA
:1028B000804B9A4201DC038000E0028048898881D5
:1028C000C88808818888C88008884880B8E62DE9CB
:1028D000F041744C6079C00722D0FCF7FEFF6066BF
:1028E000FCF7F8FAFCF7F9FF07B2A06D4FF6FF7698
:1028F00008380125A0650CE0607A012811D006EAAD
:1029000085002082A06D0838A065FCF7E3FA6D1CF5
:102910002DB2BD42F0DBA06D001DA065002020821D
:10292000B3E406EA4510ECE72DE9F0415D4C60792F
:10293000C00726D0FCF751FD6066FCF7D5FBFCF71D
:102940004CFD0646A06D4FF6FF77001F0125A065E0
:102950000CE0607A012811D007EA45002082A06DC2
:10296000001FA065FCF7C0FB6D1C2DB2B542F0DB6B
:10297000A06D001DA0650020208286E407EA0510F6
:10298000ECE7A06D0C30A0657FE42DE9F0474548E9
:102990004179C90748D0FCF720FD87B2FCF71DFD3F
:1029A00084B2FCF71AFD86B2FCF737F90546FCF74E
:1029B00014FD3C4980B2743131F81420B7FBF2F3B6
:1029C00002FB137700223A4B1EE0641EA4B2401EA5
:1029D00031F814C080B2E146B7FBFCFC31F810803E
:1029E000012C0CFB08FC33F815804CEA080C1FFA8C
:1029F0008CFC23F815C001D1012808D0B7FBF9F8E9
:102A000009FB1877521C92B2B242DED318E6B1F835
:102A1000028007F00F0202FB08F242EA0C0223F8E0
:102A20001520721C92B2EDE7816D1431816507E6C5
:102A300070B51C484079C0071DD0FCF7EEF805467C
:102A4000FCF7EBF80446FCF7E8F8194931F81520D3
:102A500031F814301A4421F8102001EB450201EB43
:102A6000440355885C8801EB40002C4444809188E5
:102A70009A881144818070BD0A4810B54179C90710
:102A800022D0FCF7CAF8C11700EB5173064901EBDD
:102A9000E30223F00703C01A044B1178083BC35C20
:102AA000194209E03000002000100020F45F000807
:102AB000001000200080FFFF03D0FC4BC05C0140F1
:102AC00000E01943117010BD816D091D816510BDB5
:102AD000F74810B54179C9071BD0FCF79EF8F549B6
:102AE000B1F8242E21F8102001EB4000B1F8222E7D
:102AF0004280B1F8202E8280B1F81E2EC280B1F83B
:102B00001C2E0281B1F81A2E4281B1F8261E818155
:102B100010BD816D091D816510BD1CB5E44841796A
:102B2000C90710D0FCF779F8E24C04EB40018A7A2F
:102B30000B7ACDE900328B790A79897834F8100064
:102B4000F1F70DFE1CBD816D091D81651CBD70B5C1
:102B5000D7484079C0071DD0FCF75FF80546FCF761
:102B60005CF80446FCF759F8D24931F8152031F8E1
:102B70001430D21A21F8102001EB450201EB440376
:102B800055885C8801EB40002C1B448091889A8812
:102B9000891A818070BD2DE9F047C5494879C2077F
:102BA0000846806D50D08946C865FCF796FE0A211C
:102BB00090FBF1F393FBF1F401FB1433642490FBDD
:102BC000F4F494FBF1F501FB15444FF47A7590FB96
:102BD000F5F595FBF1F601FB165542F2107690FBE8
:102BE000F6F696FBF1F701FB1766B34F90FBF1F297
:102BF00090FBF7F797FBF1FC01FB1C77DFF8BCC2F9
:102C000001FB120290FBFCFC9CFBF1F801FB18CCD1
:102C1000DFF8AC8290FBF8F090FBF1F801FB1800B4
:102C20000CEB0010000600EB075000EB064000EB39
:102C3000053000EB042000EB03108118C9F8641084
:102C4000BDE8F047FCF746B910308865F8E410B5E8
:102C5000974C6079C1072046806D24D0E065FCF771
:102C6000BCFB4FF47A7290FBF2F190FBF2F302FBA3
:102C70001300642290FBF2F3090341EA032190FB65
:102C8000F2F302FB13020A2392FBF3F041EA001075
:102C900092FBF3F103FB112100B208436066BDE82B
:102CA0001040FCF721BA0830A06510BD10B5804C6B
:102CB0006079C1072046806D1ED0E065FCF78DFB72
:102CC000C0F303314FF47A725143C0F3032202EB95
:102CD000C20303EB021201EB8201C0F3031202EB09
:102CE000820201EB420100F00F00084400B260666E
:102CF000BDE81040FCF7F8B90830A06510BD70B50C
:102D00006B4C6079C0071DD0FCF7E7FD0646FCF769
:102D1000E4FD464304F18805F017C5E90060FBF7C0
:102D20007CFFA16D00B2091DA16562492A8821F8C6
:102D3000102001EB40006A884280A9888180E988E0
:102D4000C18070BDA06D1830A06570BD70B5584CC5
:102D50006079C00723D0FCF7C0FD06B2FCF7BDFDCB
:102D600000B296FBF0F104F16C05296096FBF0F1DE
:102D700000FB11602E1D3060FBF74FFFA16D00B20C
:102D8000091DA1654B492A8821F8102001EB40005C
:102D90006A884280318881807188C18070BDA06D51
:102DA0001830A06570BD10B5FCF797FD0446FCF720
:102DB00094FD3F490A7B012A4A794FEA42624FEA71
:102DC00012624A7102D084420ED010BD8442FCD1FE
:102DD000088C3C4C04EBD003344C00F00700083C5A
:102DE0001B78205C0342F0D042F00100487110BD16
:102DF00010B5FCF7F2FA0446FCF7EFFA2C490A7B0F
:102E0000012A4A794FEA42624FEA12624A7102D0BD
:102E100084420ED010BD8442FCD1088C294C04EBB6
:102E2000D003224C00F00700083C1B78205C0342D2
:102E3000F0D042F00100487110BD10B5FCF74DFD17
:102E40000446FCF74AFD1A490A7B012A4A794FEAEF
:102E500042624FEA12624A7102D084420EDC10BD17
:102E60008442FCDD088C174C04EBD0030F4C00F0BF
:102E70000700083C1B78205C0342F0D042F00100C0
:102E8000487110BD10B5FCF7A8FA0446FCF7A5FA86
:102E900007490A7B012A4A794FEA42624FEA1262E5
:102EA0004A7111D084421CDC10BD0000F45F0008A0
:102EB0003000002000100020A086010040420F00DA
:102EC00080969800001000208442EDDD088CD84CDC
:102ED00004EBD003D74C00F007001B78205C0342C2
:102EE000E2D042F001004871DEE710B5FCF7F5FCD6
:102EF0000446FCF7F2FCD0490A7B012A4A794FEAE2
:102F000042624FEA12624A7102D084420DDBCBE783
:102F10008442C9DA088CC64C04EBD003C54C00F0DF
:102F200007001B78205C0342BED042F001004871CC
:102F3000BAE710B5FCF751FA0446FCF74EFABE4961
:102F40000A7B012A4A794FEA42624FEA12624A71C9
:102F500002D084420DDBA7E78442A5DA088CB44C8A
:102F600004EBD003B34C00F007001B78205C034255
:102F70009AD042F00100487196E710B5FCF7ADFC1D
:102F80000446FCF7AAFCAC490A7B012A4A794FEABD
:102F900042624FEA12624A7102D084420DDD83E739
:102FA000844281DC088CA24C04EBD003A14C00F0DD
:102FB00007001B78205C0342F1D042F00100487109
:102FC00072E710B5FCF709FA0446FCF706FA9A49CD
:102FD0000A7B012A4A794FEA42624FEA12624A7139
:102FE00002D084420DDD5FE78442FCDC088C904C0B
:102FF00004EBD0038F4C00F007001B78205C0342E9
:10300000F1D042F0010048714EE710B5FCF765FCC5
:103010000446FCF762FC88490A7B012A4A794FEA98
:1030200042624FEA12624A7102D084420DDA3BE7F3
:103030008442FCDB088C7E4C04EBD0037D4C00F01A
:1030400007001B78205C0342F1D042F00100487178
:103050002AE710B5FCF7C1F90446FCF7BEF976493A
:103060000A7B012A4A794FEA42624FEA12624A71A8
:1030700002D084420DDA17E78442FCDB088C6C4CEA
:1030800004EBD0036B4C00F007001B78205C03427C
:10309000F1D042F00100487106E710B5FCF71DFCC5
:1030A0000446FCF71AFC64490A7B012A4A794FEA74
:1030B00042624FEA12624A7102D084420DD1F3E6B5
:1030C0008442FCD0088C5A4C04EBD003594C00F0DD
:1030D00007001B78205C0342F1D042F001004871E8
:1030E000E2E610B5FCF779F90446FCF776F95249A7
:1030F0000A7B012A4A794FEA42624FEA12624A7118
:1031000002D084420DD1CFE68442FCD0088C484CDA
:1031100004EBD003474C00F007001B78205C03420F
:10312000F1D042F001004871BEE610B5424CA06DEE
:1031300010F8021BA065007801EB0022A2833F4932
:10314000E07901EB400101F5905161640A80EFF7ED
:103150002AFAE079BDE8104000F5B050FBF7FEBA5E
:1031600010B5354CE079EFF758FAE07900F5B0503A
:10317000FBF7F4FAE079BDE8104000F5C060FBF71A
:10318000EDBA10B52C4CA16D11F8020BC0F346003E
:10319000A083A16509880A0A862A02D0882A0AD152
:1031A00003E0C9B200EBC11004E0C9B200EBC110EA
:1031B00000F57A70A0836079C00716D01F49A08BF4
:1031C00001EB400000F500500288E07901EB40017E
:1031D00001F58051A1F80022EFF7E5F9E079BDE8AB
:1031E000104000F5B050FBF7B9BABDE81040B7E7A2
:1031F0001148826D12F8021BC1F34601C18382653A
:103200001288130A862B02D0882B0AD103E0D2B28F
:1032100001EBC21104E0D2B201EBC21101F57A71E7
:10322000C1834079C00701D0FEF758B8FEF700B956
:1032300000100020EC5F000830000020001000208B
:10324000DFF848C170B51CEA111E1EBF1CEA131539
:103250009EEA0C0F95EA0C0F00F06F8081EA0304E0
:1032600023EA4C134EEAD47E21EA4C1141F480113A
:1032700043F48013AE44A1FB024CA0FB0365AEF106
:103280007F7E361955EB0C05A1FB034C4CF1000376
:10329000A0FB021C16EB0C06654153F1000309422A
:1032A00018BF46F0010613F4007F0BD14FEA03313B
:1032B0004FEA0530340341EA155140EA16506FF0E9
:1032C00003020AE04FEAC3214FEAC520F40241EAB3
:1032D000555140EA56506FF0020202EB2E4201EBCC
:1032E000025585EACE710AD05FEA440C18BF24F07B
:1032F000004450F1000041F1000120EAD47040F296
:10330000FE7C624500D270BDA84214BF4FF08044DD
:103310004FF04044002E08BF0024BEF1806FA8BFCC
:10332000A1F1C041BDE87040B1F664AE4FF00000BD
:1033300001F1C04101F0004170479EEA0C0F0CEA18
:10334000131518BF95EA0C0F06D04FF0000081EA64
:10335000030E0EF0004170BDF2F7B3FD8900013E8F
:1033600000F007B800F009B84FEA430C5FEA5C5C74
:1033700008D081EA0301F1F73DBE4FEA410C5FEA54
:103380005C5CF6D14FF00000014970470000FF0778
:103390000000F87F2DE9F04101F5801CBCF5001F0D
:1033A000C0F2C3804FEA115C21EA0C510CF1FD0C14
:1033B00041F480115FEA5C0C0CF5C07C01D3400045
:1033C00049413DA4890241EA905187028E0E0A0CC0
:1033D000A45D04FB04F602FB06F6C6F14046A4FB1E
:1033E0000662F60D46EA422606FB06F4A4FB01231C
:1033F0005242C3F1404338BF5B1EA6FB0242002489
:10340000E6FB0324D20B42EA4446A6FB0623A1FBBB
:1034100002E2A3FB07E4A4184FF0000252F10002FD
:10342000E3FB01426442C2F1404E38BFAEF1010EEF
:10343000A6FB04234FF00002E6FB0E32A2FB03467C
:103440004FF00004B61954F10004E2FB0264A1FB42
:1034500006E6A4FB07E816EB08064FF0000858F153
:103460000008E4FB01687642C8F1405838BFA8F173
:103470000108A2FB06E4A3FB08E52D194FF00004A8
:1034800054F10004E2FB0854A1FB05E6A7FB04E8A5
:1034900018EB06084FF0000656F10006E1FB048623
:1034A00018F1200556F10006A809A8F11B08B1097A
:1034B00008F03F08B8F10A0F40EA86601CD901EB1A
:1034C0000C51BDE8F08100BFFCF5EEE8E2DDD8D399
:1034D000CFCBC7C3C0BDB9B6B4B1AEACA9A7A5A385
:1034E000A19F9D9B9A9896959392908F8D8C8B8996
:1034F0008887868584838281A0FB006800FB01F2B7
:1035000008EB4208B8EB872807D5341858EB0104BC
:10351000D5D5401C51F10001D1E7341A78EB0104F4
:10352000CDD4401E71F10001C9E75FEA4C0C5FEA9F
:103530009C5C0DD105D34FF0000001F00041BDE8C7
:10354000F081BDE8F04170B5F2F7BBFC6DDBFFBE6A
:10355000BDE8F0414FF00000004970470000F87FDF
:1035600010B591EA030F48BF83F0004332F522AA59
:10357000841A71EB030C07D212198CF0004C43EB48
:103580000C03001B61EB0C01DFF8A4E14FEA1154BE
:10359000A4EB135C1EEA430F18BF9EEA445F00F0E1
:1035A000B08023EA6E03524221EA0451C3EB6E035A
:1035B00038BF5B1EDCF1200E25D322FA0CFE10EB87
:1035C0000E0043FA0CFE41EB0E01CCF1200E03FA83
:1035D0000EFE10EB0E0051F10001CCF1200E29D4AB
:1035E00012FA0EF201EB0451BDE8104058BF7047CB
:1035F000401C1CBFB2F1004F704700280CBF491C93
:1036000020F00100704712EB020E43EB030218BFDB
:103610004FF0010E4EEA4202ACF1200CDCF11E0E1E
:1036200054D943FA0CFE10EB0E0051F1FF31CCF1EE
:103630001E0ED5D50EF1010E12FA0EFE404141EBE1
:10364000010101EB445C5FEA5C5C10D910EBDE70B9
:1036500001EB045138BFBEF1004FBDE8104018BF68
:10366000704700280CBF491C20F00100704730D281
:103670004FEAD42C11F5001124F400641BD0B1FAE8
:1036800081F20B3AA41AA41ED2F12003914030FA21
:1036900003F31943904001EBCC71002C01EB045172
:1036A000BDE81040A8BF704701F1C0414FF00000D5
:1036B00001F000417047B0FA80F310FA03F100D135
:1036C00010BDE41A173C4805C90AE4E701EB0451B0
:1036D00010BD491001EB0451BDE810404FEA300025
:1036E00002E04FF0000170474A0008BF0042F8D0E6
:1036F000B2F5001F28BF704701F000414FF00000F5
:1037000070479EEA445F07D011EA5E0FBDE81040A3
:1037100004BF002100207047BDE8104070B5F2F7EB
:10372000D0FB00BF40DFF63E83F0004110467047FB
:103730000000E0FF90EA010F48BF81F0004100F176
:10374000BC82421A3CBF801A89184FEAD0524FF00F
:103750007F4C1CEA410FA2EBD15318BF9CEA026FC9
:1037600000F03B804FF0004C4CEA00204CEA012175
:1037700021FA03FC10EB0C0C1ED202F1FF325FEABF
:103780001C2040EBC25038BF70471CF07F0F4FEA3F
:10379000400C18BFBCF17F4F38BF7047C3F1200306
:1037A000994008BF20F00100BCF17F4F38BF70473F
:1037B000A0F1C040F2F715BC4FEA3C00000A40EB14
:1037C000C25028BF1CF0FF0F4FEA400CE6D018BFD4
:1037D000BCF17F4F38BF7047EAE79CEA026F05D023
:1037E00010EA5C0F08BF00F00040704710B500F011
:1037F000E6F900BF64FBBE3E4FF47F0C1CEAD0121A
:103800001EBF1CEAD11392EA0C0F93EA0C0F00F0D2
:10381000858090EA010F48BF42F4807240F4000CAA
:1038200041F400002CF07F4120F07F4000B5814240
:10383000A2EB03020FF2081CACEB504EC0F10000EB
:103840009EF800E04FEA4E0E00FB0EFC38BF490028
:103850004FEA2C1C02F5FA020CFB0EF34FEACE1EC7
:103860004FEA112C4FEAC1210EEB635E42EB22427C
:103870000EFB0CFC4FEA1C5300FB03114FEA112C0A
:103880004FEA01310EFB0CFC4FEADC4C00FB0C1143
:10389000C14228BF09184CEB03335DF804EB10EB71
:1038A000410143EBC250B2F57C0F38BF704729D5B8
:1038B00012F0F00F1CBF00F1C04000F00040704754
:1038C000008182838485868788898B8C8D8E8F91F9
:1038D0009293959697999A9C9D9FA0A2A3A5A7A81D
:1038E000AAACAEB0B2B3B5B7B9BCBEC0C2C5C7C949
:1038F000CCCED1D4D7D9DCDFE2E6E9ECF0F3F7FAAD
:10390000FE0000004FEA400C0CF1807CBCF17E4FC1
:1039100028BF7047B0F1C040F2F763BB90EA010FD7
:103920000CEAD11348BF42F48072624538BF634548
:1039300007D213F47F0F16D080EA010000F0004098
:10394000704710B500F03BF9097EFC3E00F005B869
:1039500080EA010000F00040704780EA010000F0BA
:103960000040F2F73EBB12F47F0F04BF02487047DD
:1039700080EA0100F2F735BB0000C07F50EA010C7D
:1039800000F113801CF5000F58BFBCF5000F01D4E7
:103990008842704707D710F5000F58BF11F5000F88
:1039A00015D488427047894270471CF5000F04D532
:1039B000BCF5000FF7D5814270474FF0807C1CEBBF
:1039C000400F38BF1CEB410F01D28142704710B548
:1039D00000F0F5F8922449004FF000504FF080516C
:1039E000F2F7F3BAC10DD1F19E0206DB4FEA0023D4
:1039F00043F0004323FA02F07047004207D54FEA34
:103A00004001B1F1FE4F02D24FF00000704710B5F7
:103A100000F0D5F849922480002070476FEA20001A
:103A20007047000010F0004148BF4042B0FA80F3F8
:103A300010FA03F2C3F19D030BD051EAC35101EB1D
:103A40001220530638BF704700F1010008BF20F074
:103A50000100704750EA010C00F113801CF5000FC3
:103A600058BFBCF5000F01D48842704707D710F546
:103A7000000F58BF11F5000F15D4884270478942D6
:103A800070471CF5000F04D5BCF5000FF7D5814237
:103A900070474FF0807C1CEB400F38BF1CEB410F90
:103AA00001D28142704710B500F089F89224490094
:103AB0004FF000504FF08051F2F787BA4FF47F0C6F
:103AC0001CEAD0121EBF1CEAD11392EA0C0F93EA33
:103AD0000C0F00F0478090EA010F48BF42F480725B
:103AE0004FF0004C4CEA00204CEA012102EB0302AB
:103AF000A0FB0113A2F50002002918BF43F0010347
:103B00005B0028BF4FEA330342EB22425FEA132CEB
:103B10004CEBC2502EBFBCEB436FB2F57C0F70472D
:103B20004FEA036CBCF1004F08BF20F00100B2F572
:103B30007C0F38BF70470BD582F0FF0212F5803F33
:103B4000C8BF704700F1C040D8BF00F000407047C8
:103B500000F5000C5FEA4C0C48BF7047B0F1C04064
:103B6000F2F73FBA90EA010F0CEAD11348BF42F4D2
:103B70008072624538BF634504D280EA010000F0DC
:103B80000040704710B500F01AF800BF8900013EF0
:103B900000F007B800F009B85FEA410C5FEA1C6C5E
:103BA00008D080EA0100F2F71CBA5FEA400C5FEA35
:103BB0001C6CF6D14FF00040A0F5800070470EF16C
:103BC000020E2EF0030E5EF8044B244204D44FEA9A
:103BD0004102B2F17F4F11D84FEA4003B3F17F4F5A
:103BE0000CD80ED14FEAD07CB2F17F4F0CEB4C0CCD
:103BF0000CF1020C08BF4CEBD17C04E04FF0080C38
:103C000001E04FEAD17C0CEB4C0324FA03F404F0FE
:103C10000704B4F1040C06D20EEB840CBDE810408E
:103C20004CF0010C6047DFE80CF0070802024FF08F
:103C30000040A0F5800010BD0846420018BFD2F138
:103C4000807288BF00F0004010BD51EA000C00F106
:103C500013801CF5000F58BFBCF5000F01D4814242
:103C6000704707D711F5000F58BF10F5000F15D496
:103C700081427047894270471CF5000F04D5BCF59E
:103C8000000FF7D5884270474FF0807C1CEB410F46
:103C900038BF1CEB400F01D28842704780EA010018
:103CA00081EA000180EA0100FFF7FDBE90EA010F02
:103CB00048BF81F000413FF544AD421A04D882F07C
:103CC0000042A0EB020011444FEAD0524FF07F4C6B
:103CD0001CEA410FA2EBD15318BF9CEA026F4AD0F5
:103CE0004FF0004C4CEA00204CEA012121FA03FC81
:103CF000B0EB0C0C0FD412F0FE0F36D05FEA4C0084
:103D00001DD5001240EBC25038BF70471CF03F0F6A
:103D100018BF70470BE0A2F101025FEA1C2040EBE4
:103D2000C25038BF70471CF07F0F18BF7047C3F1F7
:103D30002003994014BF401E20F001007047800806
:103D40004FEA122308BF7047B0FA80FCA2EB0C02C6
:103D5000CCF1280C60FA0CF093EA122F04BF00EBB0
:103D6000C25070474FEAC3707047130A5FEADC1015
:103D700008BF7047F6E79CEA026F04D010EA5C0FB8
:103D800008BF0020704710B5FFF719FF40DFF63E6F
:103D900081F0004070470CF00F03092B08BF08208A
:103DA00000F059800A2B0BD0082B18BF704708BFB2
:103DB0001CF0400F0AD04FF000004FF00001704798
:103DC0001CF0400F18BF4FF0004070471CF0100F60
:103DD00008D020F0704300F07F4242EAD3014FEA5E
:103DE0004370704700F0604021F07F4242EA0002D9
:103DF00001F07F4040EA727070474FF0FF0C4CF4C6
:103E0000E06C1CEA11531CBF9CEA030C9445C2BF32
:103E1000DA4201EB02517047002B0DD0BCF1000FCC
:103E20000FD0002A01F00041A4BF41F0E04141F071
:103E30007F614FF00000704701F000414FF000003B
:103E4000704750EA01334FF09B0C18BF4CF0806C68
:103E500071F450AE70471CF4801F11D01CF4E02F99
:103E600003D06FEACC31490070474FF04050EFF378
:103E7000008222F0704242EA000282F3008870471A
:103E80004FF000007047C800F65E10001000000000
:103E900025001E000000FFFF0000000000000000E1
:103EA000A500A500A500A500A50011080F000A00A7
:103EB0000000000000000000000000000000000002
:103EC00000003D001C00000000001400FF00D703AC
:103ED000000000000000FFFFFFFFFFFFFFFFFFFFEC
:103EE000FFFFFFFFFFFF0000FFFF000000000000DA
:103EF00000000000000000000000000000000000C2
:103F000000003B180000000000000000000000005E
:103F10000000F401000000000000000000000000AC
:103F20000000000000000000000000000000000091
:103F30000000000000000000000000000000000081
:103F4000000000000000000000000000000064000D
:103F5000F65E1000000000000000000000000000FD
:103F60000000000000000000000000000000DC0D68
:103F7000B63D00000000000000000000000002004C
:103F8000030000000000000000000000000000002E
:103F90000000000000000000000000000000000021
:103FA0000000000000000000000000000000000011
:103FB0000000000000000000000000000000000001
:103FC00000000000000000000000000000000000F1
:103FD00000000000000000000000000000000000E1
:103FE00000000000000000000000000000000000D1
:103FF00000000000000000000000000000000000C1
:1040000000000000000000000000000000000000B0
:1040100000000000000000000000000000000000A0
:104020000000000000000000000000000000000090
:104030000000000000000000000000000000000080
:104040000000000000000000000000000000000070
:104050000000000000000000000000000000000060
:104060000000000000000000000000000000000050
:104070000000000000000000000000000000000040
:104080000000000000003031323334353637383923
:10409000414243444546000000000000000000008B
:1040A0000000000000000000000000000000000010
:1040B0000000000000000000000000000000000000
:1040C00000000000000000000000000102030405E1
:1040D00006070809000000000000000A0B0C0D0E86
:1040E0000F00000000000000C1814001C0804101BC
:1040F000C0804100C1814001C0804100C1814000B9
:10410000C1814001C0804101C0804100C1814000A7
:10411000C1814001C0804100C1814001C080410196
:10412000C0804100C1814001C0804100C181400088
:10413000C1814001C0804100C1814001C080410176
:10414000C0804100C1814000C1814001C080410167
:10415000C0804100C1814001C0804100C181400058
:10416000C1814001C0804101C0804100C181400047
:10417000C1814001C0804100C1814001C080410136
:10418000C0804100C1814000C1814001C080410127
:10419000C0804100C1814001C0804100C181400018
:1041A000C1814001C0804100C1814001C080410106
:1041B000C0804100C1814001C0804100C1814000F8
:1041C000C1814001C0804101C0804100C1814000E7
:1041D000C1814001C0804100C1814001C0804101D6
:1041E000C0804100C1814000C0C101C30302C2C6FA
:1041F0000607C705C5C404CC0C0DCD0FCFCE0E0AE3
:10420000CACB0BC90908C8D81819D91BDBDA1A1E82
:10421000DEDF1FDD1D1CDC14D4D515D71716D6D252
:104220001213D311D1D010F03031F133F3F2323612
:10423000F6F737F53534F43CFCFD3DFF3F3EFEFA22
:104240003A3BFB39F9F83828E8E929EB2B2AEAEE62
:104250002E2FEF2DEDEC2CE42425E527E7E6262292
:10426000E2E323E12120E0A06061A163A3A26266F2
:10427000A6A767A56564A46CACAD6DAF6F6EAEAA62
:104280006A6BAB69A9A86878B8B979BB7B7ABABE02
:104290007E7FBF7DBDBC7CB47475B577B7B67672D2
:1042A000B2B373B17170B0509091519353529296D2
:1042B000565797559594549C5C5D9D5F9F9E5E5AA2
:1042C0009A9B5B99595898884849894B8B8A4A4EE2
:1042D0008E8F4F8D4D4C8C44848545874746868212
:1042E000424383418180401F1C1F1E1F1E1F1F1E33
:1042F0001F1E1F00000000004C5555555555A53F89
:104300007751C1166CC156BF9015CB19A001FA3E6A
:10431000AD529C804F7E92BEC4B1B4BD9EEE213E94
:10432000D43888BEE9FAA8BD00004054FB21F93F0B
:104330003163621A61B4D03D0000601A61B4D03DAF
:104340007370032E8A19A33B0000002E8A19A33B29
:10435000C14920259A837B3900000000000000003D
:104360006E83F9A22915444ED15727FCC0DD34F5E0
:10437000999562DB4190433CAB6351FE61C5BBDE66
:104380003A6E24B7E0D24D42EA2E49061C92D1097A
:104390001CEB1DFE3EA729B1F53582E88444BB2EF7
:1043A00026709CE9417E5FB439D69139F439538344
:1043B0008B5F849C3B28F9BDFF97F81F0F9805DEA3
:1043C0008B112FEF1F6D0A5ACF7E366DB709CB27A1
:1043D000663F464F2DEA5F9EC7BA27757BF1E5EB36
:1043E000F739073DEA92528AB15FFB6B085D8D1F7A
:1043F000A6F810111111813FD561C119A0012ABF82
:104400007DFEB157E31DC73EEB9C2B8AE6E55ABE05
:104410007CD5CF5A3AD9E53D7AFE10111111C13F32
:1044200037D60684F464963F280356C9226D6D3F43
:104430000165F2F2D844433FA69237A0887E143F2C
:10444000735360DBCB75F3BEFE41B31BBAA1AB3F28
:1044500093846EE9E326823F1583E0FEC8DB573F75
:1044600068108D1AF726303FE9A7F0320FB8123FD7
:10447000D47ABF74702AFB3E9844010800000020E3
:10448000240100005C010008BC4501082401002053
:10449000C4D40000780100080204060800000000EF
:1044A00001020304010203040607080900A24A04EA
:1044B00000000000000000000102030406070809D4
:1044C0000000000000000000FF00000000000000ED
:1044D00000000000000000000000000000000000DC
:1044E00000000000000000000000000000000000CC
:1044F00000000000000000000000000000000000BC
:1045000000000000000000000000000000000000AB
:10451000000000000000000000000000000000009B
:10452000000000000000000000000000000000008B
:10453000000000000000000000000000010010006A
:10454000000100100000000000000000000000005A
:1045500000000000000000000100030007000F0041
:104560001F003F007F00FF00FF01FF03FF07FF0F59
:10457000FF1FFF3FFF7FFFFF000000000000000063
:1045800000000000000000000A0000000100000020
:10459000010000000000000000000000000000001A
:1045A000000000000000000000000000000000010A
:0C45B000040400020500030601040600DC
:0400000508000121CD
:00000001FF
